:020000040000FA
:10000000E0700020E1000000E9000000D5000000E1
:1000100000000000000000000000000000000000E0
:10002000000000000000000000000000ED000000E3
:100030000000000000000000EF000000F1000000E0
:10004000F3000000B16C0000216C0000F300000020
:1000500005160000F3000000F3000000F3000000AC
:10006000F3000000F300000059700000F3000000EE
:10007000F3000000F300000071700000F3000000C6
:10008000F3000000F300000000000000F300000097
:1000900079630000F3000000F3000000251A00005F
:1000A000D1130000F3000000F3000000691300000A
:1000B000F3000000F3000000F3000000F300000074
:1000C0000348854600F0DAFC004800472D8B00000D
:1000D000E07000207046694608F0B6FAFFF7FEFFB0
:1000E0000448804704480047FEE7FEE7FEE7FEE7D6
:1000F000FEE7FEE76D6E0000C100000030B50B4664
:10010000014600202022012409E00D46D5409D42F1
:1001100005D31D469540491B254695404019154677
:10012000521E002DF1DC30BD70B50024254600289C
:1001300001DA01244042002901DA01254942FFF792
:10014000DDFFAC4200D04042002C00D0494270BDDF
:10015000F0B51FB40646002082B005464024019148
:1001600000901BE0019922460F46304600F0C2FB8A
:10017000049A059B801A994110D3104619462246CD
:1001800000F0A8FB361A8F4101972246012000217A
:10019000009F00F09FFB38184D4100902046641EE0
:1001A0000028DFDC019B00982946324607B0F0BDED
:1001B00003460B439B0703D009E008C9121F08C080
:1001C000042AFAD203E00B780370401C491C521E2B
:1001D000F9D27047D2B201E00270401C491EFBD236
:1001E00070470022F6E710B513460A460446194642
:1001F000FFF7F0FF204610BD30B505462A460B46F6
:1002000010781C78521C5B1C002801D0A042F7D04B
:10021000002C03D0002802D06D1CEFE7284630BD2B
:10022000421C0178401C0029FBD1801A7047032131
:10023000001D401E037812021A43491EF9D51046CC
:100240007047034603220870000A491C521EFAD563
:1002500018467047F8B502464A40D40F42004B009A
:1002600052085B089A4202D20246084611464A00EA
:1002700023D0C30D4A00DDB2120EAD1A202D35DA9F
:1002800049020126490AF6058A19002C00D052427B
:1002900020214F1B1146B9402A411018C20D9A4225
:1002A00021D0002C17D0012D08DCDA05801AD20FDE
:1002B0008019D207DBB200F049FBF8BDDA05801ADD
:1002C000012340001B06C01880185A428018CA0F2C
:1002D0001043490007E04908C2071143DA05801AB4
:1002E00080194008801800F029FBF8BD6100012248
:1002F000511A001BF7E70122D2075140AAE7012259
:10030000D2075040A6E7024670B54A40D30FDB073C
:1003100040002DD04A002AD0010E140E0002120215
:100320000919400A520A8418E50104465443000A98
:10033000120A2E045043A4194219200CC543AA18CE
:10034000120C0125AD03521C521912047F392404EA
:1003500000D0521C104301D44000491EC2B20C060A
:10036000C0092018401C4008802A02D003E0002069
:1003700070BD40084000002900DA0020184370BD1D
:1003800070B502464A40D50F40004A00ED074008CC
:100390005208002814D0002A12D0C40DD30D4102F7
:1003A0000120C0055202490A520AE41A091812181B
:1003B0007D34914201D3641C00E04900002C01DA35
:1003C000002070BD0023914201D3891A03434008E5
:1003D00049000028F7D100290AD0914202D1012119
:1003E000C90705E0914201D2012101E00121C94381
:1003F000E005C018401900F0A1FA70BDF0B507463D
:100400000846584087B0C00F049048000E46590077
:1004100040084908BC1A884105D2384631461E4674
:1004200017460B4602465800400810434CD0300D8A
:10043000039040055900400D490D0590401A029067
:10044000402872DA18030121000B090508430190C6
:1004500004980092002805D001995242002088415A
:1004600000920190029840210A1A0199009800F028
:1004700031FA05460C466B4607CB00F04CFAC01922
:100480007141039A0E0D0023D71756401A467A4041
:10049000164344D0049A002A2DD0029A012A039AC6
:1004A00015DC1205C01A914101263605001C714168
:1004B000D20F059ED2070093019202962A46234648
:1004C00000F08AFA07B0F0BD38463146FAE7160563
:1004D000224A0F46B218C01AB74101210905001C73
:1004E0004F4100187F41114618187941E20F10431F
:1004F0006D19644113E0E2076D0815436408C207F3
:100500001443039A01261205C01A91413605001CB6
:100510007141CE07400830434908C01851412A466E
:10052000234600F04CFACDE7FFE704980122400093
:10053000C117121A00238B4104983146C417381A88
:10054000A141EEE730B40124E407634030BC55E735
:1005500030B40124E407614030BC4FE70000E0FF05
:10056000F0B51FB488B00B99099800244840099948
:10057000C00F490049080991C0070B990090490034
:1005800049080B9109990898A64608431CD00B9975
:100590000A98084318D0099801244000420D4800E9
:1005A000410D099824050003000B204309900B9886
:1005B0000003000B20430B9050181C4940180022E8
:1005C00001901446104605E0002001460DB0F0BD34
:1005D000032801DA034600E003239C46C11A0AAE51
:1005E0000AE05F0008ADED5B4F00F75B7D4300273D
:1005F000AA187C41491C5B1E6145F2DD410004AB39
:100600005A522104120C0A43240C401C0828DFDB38
:10061000019802900099704601910090059B049A00
:100620000799069800F0D8F9D0E700000DFCFFFF0D
:10063000F0B50C465C4085B0E40FE40703944C0031
:10064000002664085900944649080246029622434F
:1006500021D062460A431ED06200570D4A000E03A5
:100660002303550D012402462C492405781B1B0B3E
:10067000360B401823432643614600901C46501A0F
:10068000B44103D30098401C009002E092180098F7
:100690005B41002803DA0020014605B0F0BD0020D0
:1006A000012109050746864611E064461D46141BD4
:1006B000B54106D36546521BB341744607430C430C
:1006C000A646CD0740084908284392185B410546D5
:1006D0000D43EAD11046184313D0604619465040E6
:1006E0007140084306D06046101AB34106D2012279
:1006F000002306E000220123DB0702E00122D243AF
:100700005310009874460105381C6141029C039DFA
:100710000019694100F053F9BFE70000FD03000034
:1007200010B500229623114600F010F910BD00000C
:100730000EB5C217C10F5040CA0740180021054B23
:100740000293019200910A460B4600F045F903B06E
:1007500000BD0000330400000EB5054902910021E0
:1007600000910A460B46019100F036F903B000BD36
:100770003304000070B5CD0F4A0009030123090BB3
:100780001B0519430B4BED070024520D9A4201DA69
:10079000002070BD074B34339A4203DC9A1A00F0F4
:1007A000A9F802E00449511888402C43F1D0404296
:1007B00070BD0000FF030000CDFBFFFF4A000903EE
:1007C0000123090B1B051943094B10B5520D9A4221
:1007D00001DA002010BD064B34339A4203DC9A1A2A
:1007E00000F088F810BD03495118884010BD000082
:1007F000FF030000CDFBFFFF4A0009030123090BA3
:100800001B0519430A4B10B5520D9A4202DA00201B
:10081000014610BD064B34339A4203DC9A1A00F0AD
:1008200069F810BD034BD21800F054F810BD000059
:10083000FF030000CDFBFFFFC20FD20740004008BE
:100840000BD0C10D0723DB01C91840020905400A7E
:100850001143C2084007114370470020014670470A
:1008600010B5002904DB0124E40740428C412146F5
:10087000002B04DB1C460123DB075242A3419942B3
:1008800000D1904210BD0000CB0FDB07490010B52E
:10089000490802460A4307D00A0D07240903E40168
:1008A000090B121B002A01DC002010BDC900440FF7
:1008B0000C43C100E018D205801800F03FF810BDCD
:1008C0000122D207002800DB101A002900DB511A90
:1008D0008842704710B5202A04DB0146203A914037
:1008E000002010BD914020239C1A0346E340194389
:1008F000904010BD10B5202A04DB0846203AD040B5
:10090000002110BD0B46D340D0402024A21A9140B4
:100910000843194610BD10B5202A06DBCB17084640
:10092000203A1041C1170B4306E00B461341D0405B
:100930002024A21A91400843194610BD002904DA68
:10094000401C490001D140084000704770B40024A9
:10095000050C05D11024000402D1002921D0112456
:10096000050E01D100020834050F01D10001241D3C
:10097000850F01D18000A41C002801DB4000641C0D
:10098000002908D020252E1B0D46F540A14000D09F
:1009900001212943084301061B1B000ADB1D02D568
:1009A000002070BC7047DB05181880180029F8DAA1
:1009B000401C4900F5D170BC40084000704710B59C
:1009C000002B08DA0024401C614192185B411A4355
:1009D00001D14008400010BDF0B51FB482B00546FB
:1009E0000C0003D0084606F045FF02E006F042FF87
:1009F00020300246009021462846FFF76BFF049BFB
:100A0000059A04460F4618431143084314D018466C
:100A100010431BD0009840210A1A18460599FFF789
:100A200069FF05460E46009A05990498FFF752FFA4
:100A3000084305D0012004E02046394607B0F0BD48
:100A40000020C11705430E432C43374300990E98ED
:100A50006305401A7905E40A00220C43FD0A0A30B6
:100A600002D500200146E9E70105101969410C9CF7
:100A70000D9D00196941FFF7A2FFDFE7064C012534
:100A8000064E05E0E36807CC2B430C3C9847103436
:100A9000B442F7D3FFF718FBC49B0000E49B0000AF
:100AA00070B58C180578401C6B075B0F01D103787B
:100AB000401C2A1106D10278401C03E006780E7013
:100AC000401C491C5B1EF9D12B0705D40023521E84
:100AD0000DD40B70491CFAE70378401CCB1A921C0A
:100AE00003E01D780D70491C5B1C521EF9D5A14214
:100AF000D8D3002070BD00000146064A10690723C4
:100B00001B0402469A4310461A460A401043014A03
:100B10001061704700FA0140012806D106490969B1
:100B200020221143044A116105E00349096920228A
:100B30009143014A1161704700FA01400146054A9C
:100B40001069000900010A07120F1043014A1061E1
:100B50007047000000FA0140012806D106490968E3
:100B600040221143044A116005E00349096840220C
:100B70009143014A1160704700FA0140012806D1F3
:100B80000649096801221143044A116005E003493E
:100B9000096849084900014A1160704700FA01409C
:100BA0000146064A1068082302469A431046082266
:100BB0000A401043014A10607047000000FA0140EB
:100BC0000146064A1068042302469A43104604224E
:100BD0000A401043014A10607047000000FA0140CB
:100BE000012806D10649096802221143044A11600E
:100BF00005E00349096802229143014A11607047E8
:100C000000FA01400148806880B2704700FA014054
:100C100010B5012000F048FC06F0D6FD012006F0DA
:100C2000E5FD022006F0C0FD012006F0ABFD0A2024
:100C3000FFF784FF0120FFF76FFF0420FFF7C0FFDD
:100C40000120FFF7CDFF01208004FFF755FF0020B2
:100C5000FFF7A6FF044800F04DF80020FFF77CFFE7
:100C60000020FFF78BFF10BDFF07000010B501202B
:100C700000F01AFC06F0A8FD012006F0B7FD0220E6
:100C800006F092FD012006F07DFD0520FFF756FFDE
:100C90000120FFF741FF0420FFF792FF0120FFF73B
:100CA0009FFF01208004FFF727FF0020FFF778FF58
:100CB000044800F01FF80020FFF74EFF0020FFF768
:100CC0005DFF10BDFF0700000548C068FF2101312E
:100CD0000840002801D0012070470020FCE70000F8
:100CE00000FA0140FF2001300149C8607047000050
:100CF00000FA01404105490D014A5160704700006A
:100D000000FA014010B5012000F0CEFB06F05CFDBA
:100D1000012006F06BFD022006F046FD012006F0E2
:100D200031FD0F20FFF70AFF0120FFF7F5FE042039
:100D3000FFF746FF0120FFF753FF0748FFF7DAFFF1
:100D400001208004FFF7D8FE0020FFF705FF0020F8
:100D5000FFF714FF10BD0000FF07000070B5054647
:100D60000E4614462946204600F088FB04480460DD
:100D70000448066002F012FD02F02EFA70BD000079
:100D8000340400203804002010B50121074800F089
:100D9000EDFC022000F0F6F94021054800F0C9F909
:100DA00001224021024801F024FC10BD070000018F
:100DB000400D004010B501231A4604210D4801F0F2
:100DC000B9F901231A4608210A4801F0B3F90123B1
:100DD0001A4619460748803001F0ACF91E2005F08C
:100DE000EFFC02211E2005F003FD1E2005F0F4FC9F
:100DF00010BD0000400C004030B50246002018E055
:100E0000002112E0130184001B195B180A4CE35CFB
:100E100084000A4D2D686419645C63408400074DAA
:100E20002D68641963544B1CD9B20429EADB431CB6
:100E3000D8B20428E4DB30BDE817002034040020D9
:100E4000F8B505460E46002E22D02868002800D1AD
:100E5000F8BD2C6801E0274664686068002802D06D
:100E60002088B042F7D12088B04210D109480078DC
:100E7000401E084908702868A04202D160682860B6
:100E800001E060687860204607F00AFE002400BF99
:100E900000BFDDE72C04002010B50121794800F0E7
:100EA00065FC0022FF210131774805F0DDFC0022BE
:100EB00080217548403005F0D7FC0022402172485F
:100EC000403005F0D1FC012291036F48803002F0E0
:100ED00006F90122D1036C48803002F000F90122AA
:100EE00051026948403002F0FAF80022012109035A
:100EF0006548803805F0B8FC00220121C90262482B
:100F0000803805F0B1FC012109035F48803801F009
:100F100064FB0121C9025C48803801F05EFB0022BD
:100F20000121C9035848803805F09EFC0121C903FE
:100F30005548803801F051FB0022012189035248B5
:100F4000803805F091FC012189034F48803801F079
:100F500044FB0022012149034B48803805F084FC02
:100F6000012149034848803801F037FB002108205F
:100F700002F0F0F800220221434802F0B0F800220B
:100F800001214148C03805F06FFC002202213E4893
:100F9000C03805F069FC002204213B48C03805F048
:100FA00063FC002208213848C03805F05DFC0022AF
:100FB00001213548803005F057FC0121324880304E
:100FC00001F00DFB002220212F4802F088F80022BA
:100FD00010212D4802F083F8012204212A4880388C
:100FE00002F07DF8012208212748803802F077F8C6
:100FF000012251032448C03802F071F80022102168
:101000002148803005F030FC002208211E48803045
:1010100005F02AFC012211461B4802F060F800216D
:10102000012002F097F80022FF2101311648803894
:1010300005F01AFC0022012149021348803805F00E
:1010400013FC002204211048C03005F00DFC0022E2
:1010500008210D48C03005F007FC0022012149039A
:101060000948403802F03BF8002280210648C03091
:1010700002F035F8002220210348803002F02FF8DA
:1010800010BD000007000001C00C00407FB50646FF
:101090000D4614466A462946304601F097F90098F5
:1010A000A84227D16846C079002823D1E007C00FA5
:1010B000002803D16846407900281BD1E007C00F03
:1010C000002803D068464079012813D1022020402F
:1010D000002803D16846807900280BD102202040E7
:1010E000002803D068468079012803D1684600793A
:1010F00002281DD0029500206946C873E007C00F82
:10110000002801D1487302E001206946487302209B
:101110002040002802D16946887302E00120694618
:10112000887302206946087302A9304601F012FA5A
:101130007FBD7FB505460C466A462146284601F02C
:1011400045F90098A0420FD16846C07900280BD11C
:1011500068464079002807D168468079002803D185
:101160006846007903280BD0029400216846C173B9
:10117000417381730321017302A9284601F0EAF942
:101180007FBD000070B505460024002600F080F900
:10119000002802D1012000F087F9002416E0012088
:1011A000A04006462846304000280ED00C48006873
:1011B0000121A14088430A4908600846816862000D
:1011C00003209040014306488160641C042CE6D350
:1011D00000F05EF9012802D1002000F065F970BD31
:1011E00000FC014000B587B0684600F069F90BA02B
:1011F00006F01CFB17A006F019FB1EA220A123A0DD
:1012000006F014FB2AA0009906F010FB03A006F0DC
:101210000DFB0FA006F00AFB07B000BD2F2A2A2AFB
:101220002A2A2A2A2A2A2A2A2A2A2A2A2A2A2A2A1E
:101230002A2A2A2A2A2A2A2A2A2A2A2A2A2A2A2A0E
:101240002A2A2A2A2A2A2A2A2A2A2A2A2A2A2A2FF9
:101250000D0A00002F6170706C69636174696F6EB4
:1012600056657273696F6E2073746172742F0D0A04
:101270000000000031313A32303A333200000000D1
:101280004A756E2031332032303234004275696C39
:10129000642044617465202020202020202020200C
:1012A0002020203D2025732025730D0A000000001A
:1012B00053797374656D20436C6F636B2046726560
:1012C0007175656E63793A20256C7520487A0A003D
:1012D0000149C8627047000000600140012806D142
:1012E0000649096880221143044A116005E0034958
:1012F000096880229143014A1160704700600140F3
:10130000012806D10649096801221143044A1160E7
:1013100005E00349096849084900014A116070471E
:10132000006001400146064A1068082302469A43BD
:10133000104608220A401043014A1060704700001E
:1013400000600140012806D10649C9680122114305
:10135000044AD16005E00349C96849084900014AC7
:10136000D16070470060014010B500F00DF8002812
:1013700006D004480068401C0249086000F010F8DC
:1013800010BD0000B003002004480069C007C00F72
:10139000002801D0012070470020FCE700600140D8
:1013A00001200149086170470060014001498862DD
:1013B0007047000000600140012904D102688023C9
:1013C0001A43026003E0026880239A430260704778
:1013D00010B51D4800F042F8012809D11A4800F064
:1013E0004AF8194800F044F801201849487029E0EB
:1013F0001548443000F032F8012823D11248443017
:1014000000F039F81048443000F032F81048007805
:10141000401C0F49087005210D480078FEF784FE36
:1014200000290FD101200B4908700B480078401C9F
:10143000C0B209490870032804DB00210248443087
:10144000FFF7BAFF10BD0000003001403C0400204F
:1014500004000020FA0000200A0100200146086C68
:1014600010221040002801D0012070470020FCE726
:101470001021016470470821016470470246002072
:1014800003E00B5C1354431CD8B21028F9DB7047FF
:10149000044800680007000F0A2801D101207047A6
:1014A0000020FCE700E00140012803D10A21034AA3
:1014B000116002E00521014A1160704700E001401F
:1014C00000B5024600230020D0601061106050601B
:1014D000906000F0B5F9012807D100F099F90346B2
:1014E0001B0C581C3B494843D06000F073F901289D
:1014F0000ED100F083F903461B0C581C36494843B3
:10150000106100F073F9082802D1106940001061E1
:1015100000F00EFA034600BF002B06D0012B07D0C7
:10152000022B08D0032B0DD108E0D06810600CE02E
:101530002A48106009E01069106006E00120C0032D
:10154000106002E0D068106000BF00BF00F0ACF98E
:1015500003461B0A042B06D0052B08D0062B0AD005
:10156000072B10D10BE01068400850600EE01068A7
:10157000800850600AE01068C008506006E01068FB
:101580000009506002E01068506000BF00BF00F02A
:10159000A3F903461B0C042B06D0052B08D0062B01
:1015A0000AD0072B10D10BE05068400890600EE085
:1015B0005068800890600AE05068C008906006E0BB
:1015C00050680009906002E05068906000BF00BF62
:1015D00000BD000000127A0040420F00001BB7005F
:1015E000012806D10649896901221143044A916103
:1015F00005E00349896949084900014A916170473A
:1016000000240040704700000548C069FF210131F7
:101610000840002801D0012070470020FCE70000AE
:101620000024004010B50446012C02D11148036883
:1016300013E0022C03D10F484038C36B0DE0032C9C
:1016400003D10C484038836B07E0042C03D10948D0
:101650004038436B01E007480368180CD94389B24E
:10166000884203D1D8B200F009F902E06B2000F003
:1016700005F910BD40FBFF1F012806D10749096B82
:1016800002051143054A116306E00449096B012272
:1016900012059143014A1163704700000024004085
:1016A000012806D10749096B02021143054A11635B
:1016B00006E00449096BFF2201329143014A11639C
:1016C00070470000002400400146054A106B800866
:1016D00080008A07920F1043014A10637047000090
:1016E00000240040012806D10749096B420211433A
:1016F000054A116306E00449096B01225202914335
:10170000014A116370470000002400400146064A68
:10171000106B0C2302469A4310460C220A401043D9
:10172000014A10637047000000240040012806D1E0
:101730000649496B10221143044A516305E00349ED
:10174000496B10229143014A5163704700240040C5
:101750000146054A506B800880008A07920F1043AB
:10176000014A5063704700000024004030B5024633
:101770000B4600200F2424061440FF252D06641973
:10178000002C09D06419002C08D06419002C08D052
:101790006419002C0BD107E00D4809E00C48001D2E
:1017A00006E00B48083003E009480C3000E000BFB9
:1017B00000BF00280BD092B201219140002B03D032
:1017C00004680C43046002E004688C43046030BD8C
:1017D0002024004004480069C007C00F002801D041
:1017E000012070470020FCE7002400400248006907
:1017F00008210840704700000024004002480069AA
:101800000249084070470000002400400000FF0328
:10181000024840680F210904084070470024004036
:101820000146064A50680F231B0402469A4310469D
:101830001A460A401043014A506070470024004095
:1018400004484068C007C00F002801D0012070473D
:101850000020FCE700240040012806D10649496821
:1018600001221143044A516005E0034949684908CF
:101870004900014A51607047002400400146044A73
:101880009068000A0002CAB21043014A9060704793
:101890000024004010B504462068FFF7C1FF2079FE
:1018A000FFF7DAFF10BD00000248006807210902B7
:1018B00008407047002400400146064A106807238C
:1018C0001B0202469A4310461A460A401043014A38
:1018D0001060704700240040024800680721090496
:1018E00008407047002400400146064A106807235C
:1018F0001B0402469A4310461A460A401043014A06
:101900001060704700240040012806D1074909688B
:1019100042061143054A116006E0044909680122A4
:1019200052069143014A11607047000000240040B4
:10193000024800684007400F704700000024004044
:101940000146054A1068C008C0004A07520F1043FC
:10195000014A1060704700000024004010B50446A2
:101960002068FFF7EDFF6068FFF7A6FFA068FFF7AC
:10197000BBFF207BFFF7C8FF10BD0000012806D188
:101980000649496901221143044A516105E00349AE
:10199000496949084900014A5161704700240040E3
:1019A0000146064A506907231B0202469A43104625
:1019B0001A460A401043014A506170470024004013
:1019C00005480068012149020840002801D0012093
:1019D00070470020FCE7000000540140012806D1B8
:1019E0000649896880221143044A916005E0034951
:1019F000896880229143014A9160704700540140F8
:101A0000012806D10649896840221143044A9160A1
:101A100005E00349896840229143014A916070477B
:101A20000054014010B500F015F801280CD100F069
:101A30001DF8FFF7C5FF012803D104A005F0F6FE4D
:101A400002E003A005F0F2FE10BD0000310D0A0017
:101A5000320D0A000448C068C007C00F002801D03A
:101A6000012070470020FCE700540140012001499B
:101A7000C860704700540140F8B504460E46002582
:101A80000027FFF705FD002802D10120FFF70CFD1C
:101A9000002512E00120A8400746304638400028C3
:101AA0000AD020680121A94088432060A1686A000B
:101AB000032090408143A1606D1C042DEAD3FFF701
:101AC000E7FC012802D10020FFF7EEFCF8BD70B55D
:101AD0000A460021002300BF12E001248C40234667
:101AE00014461C40002C0AD0046801258D40AC43EC
:101AF0000460C4684E000325B540AC43C460491C73
:101B00001029EAD370BD032001218907486070477E
:101B10000146064AD069131502469A4310461A46F2
:101B20000A401043014AD061704700004004004061
:101B3000012806D10649C96901221143044AD1612D
:101B400005E00349C96949084900014AD161704764
:101B5000400400400146064AD069931502469A4364
:101B600010461A460A401043014AD06170470000EF
:101B700040040040012806D10649C96904221143E6
:101B8000044AD16105E00349C96904229143014A2D
:101B9000D161704740040040012806D10649C96957
:101BA00002221143044AD16105E00349C9690222B6
:101BB0009143014AD1617047400400400146064A02
:101BC000D06903231B0302469A4310461A460A4073
:101BD0001043014AD0617047400400400146064A64
:101BE000D069531502469A4310461A460A401043DC
:101BF000014AD06170470000400400400004054ADB
:101C0000D169054A1140D24302401143014AD161D2
:101C10007047000040040040FFFF00E0C103490C92
:101C2000014A1162704700004004004030B502468E
:101C3000D400064D6319186830250446AC4320468D
:101C400030240C402043186030BD000004040040E4
:101C500010B50246D300074C1819012904D10424F9
:101C600003682343036003E004240368A343036081
:101C700010BD00000404004010B50246D300074C1C
:101C80001819012904D1022403682343036003E0E7
:101C900002240368A343036010BD00000404004055
:101CA00030B50246D400064D63191868ED14044699
:101CB000AC4320462C460C402043186030BD000049
:101CC0000404004030B50246D400064D631918687C
:101CD00003252D030446AC4320462C460C402043EC
:101CE000186030BD0404004030B50246D400064DF3
:101CF0006319186807252D020446AC4320462C467C
:101D00000C402043186030BD0404004030B502464A
:101D1000D400054D631909041868044C2040E443BD
:101D20000C402043186030BD04040040FFFF00E079
:101D300010B50246D300074C1819012904D1082414
:101D400003682343036003E008240368A34303609C
:101D500010BD00000404004010B50246D300074C3B
:101D60001819012904D1012403682343036003E007
:101D700003685B085B00036010BD000004040040C2
:101D800030B50246D400064D631918684025044654
:101D9000AC43204640240C402043186030BD000076
:101DA000040400400146C800014BC2181068704787
:101DB0000804004010B5C300014C1A19116010BD91
:101DC00008040040012806D1064909680122114390
:101DD000044A116005E00349096849084900014ABD
:101DE0001160704700040040012109048140014A4C
:101DF000916270474004004010B5044620780B28DB
:101E000023D120780021FFF7A7FF6068FFF7F6FED7
:101E1000A068FFF7D3FE6069FFF77AFE606AFFF7FC
:101E2000DDFEA06AFFF796FE607FFFF7A3FEA07FAE
:101E3000FFF7B2FE2078216AFFF7BCFFE06AFFF7E8
:101E4000EDFEE07FFFF774FE2FE020780021FFF722
:101E500083FF20786168FFF759FF2078A168FFF7BA
:101E600031FF2078E168FFF71BFF20782169FFF739
:101E70003BFF20786169FFF783FF2078A169FFF7B6
:101E8000D5FE217F2078FFF753FF617F2078FFF791
:101E9000DFFEA17F2078FFF7EFFE2078216AFFF7B1
:101EA00089FFE17F2078FFF757FF10BD00B585B0AF
:101EB0000020FFF795FB0020FFF760FD0120FFF7F2
:101EC000F3FA012004F048FE002004F035FE012062
:101ED00004F020FE002005F089FC0020FFF7E4FA62
:101EE00002200090000201900020694608720390D1
:101EF00003200490684604F01FFD01F05DF801F036
:101F000063F830BF01F058F8002004F003FE05B07C
:101F100000BD00000146054A1068800880008A075D
:101F2000920F1043014A10607047000000100040FB
:101F300001460020044A12690A40002A01D001200B
:101F400000E000207047000000FC0140F7B50346A8
:101F50000D460021002207E0012696402E40002E6B
:101F600001D0114602E0521C102AF5D300BF102AFE
:101F700000D1FEBD314FDE1BBB4211D008DC304E1C
:101F80009E19002E09D0402E08D0802E51D106E097
:101F9000402E06D0802E4CD104E000BF00BF00BF11
:101FA00000BF00BF254E4036B34203D0234E8036DB
:101FB000B34202D10B2903D93CE00F2900D939E003
:101FC000032901D800200CE0042903D3072901D8F4
:101FD000012006E0082903D30B2901D8022000E0E4
:101FE0000320164E803EB34200D1001D134E403EEA
:101FF000B34200D10830114EB34200D10C300F4E25
:102000004036B34200D110300C4E8036B34200D17E
:1020100014300C4E3469029E012E02D186403443A6
:1020200004E0012686402746B7433C46054E34610E
:1020300000E000BF00BF00BF9BE70000C00C0040F5
:1020400000F4FFBFC00D0040F0B502460C46002171
:10205000002307E001269E402640002E01D01946AD
:1020600002E05B1C102BF5D300BF102B00D1F0BD9C
:102070002D4FD61BBA4211D008DC2C4E9619002EDB
:1020800009D0402E08D0802E49D106E0402E06D03F
:10209000802E44D104E000BF00BF00BF00BF00BFDE
:1020A000214E4036B24203D01F4E8036B24202D19A
:1020B0000B2903D934E00F2900D931E0032901D8D5
:1020C00000200CE0042903D3072901D8012006E0F1
:1020D000082903D30B2901D8022000E00320124E67
:1020E000803EB24200D1001D0F4E403EB24200D1B0
:1020F00008300D4EB24200D10C300B4E4036B24289
:1021000000D11030084E8036B24200D11430084E53
:102110007569012686403540054E756100E000BFB7
:1021200000BF00BFA3E70000C00C004000F4FFBFE9
:10213000C00D0040F8B505460E4617461C46032262
:102140003146284600F022F83146284600F0A4F82F
:10215000224631462846FFF7F9FE3A4631462846E0
:1021600000F014F8C82006F0D9FB31462846FFF7E6
:102170006BFF1E20002805DBC206D20E0121914014
:10218000014A116000BFF8BD80E200E0F7B50346E8
:1021900015460021002408E00126A640019F3E408C
:1021A000002E01D0214602E0641C102CF4D300BFA5
:1021B000102C00D1FEBD354FDE1BBB4211D008DC18
:1021C000334E9E19002E09D0402E08D0802E58D1B3
:1021D00006E0402E34D0802E53D132E000BF00BF45
:1021E00000BF0F2900D94DE0032901D800200CE0E1
:1021F000042903D3072901D8022006E0082903D3C4
:102200000B2901D8042000E00620204E803EB34276
:1022100000D108301D4E403EB34200D110301B4E5D
:10222000B34200D118301B4EB268032686401746D1
:10223000B7433A462E4686403243164EB26021E0FE
:1022400000BF0B2900D91DE0032901D8002006E0BA
:10225000042903D3072901D8022000E004200B4EF3
:102260008036B34200D108300A4EF2680326864019
:102270001746B7433A462E4686403243054EF26033
:1022800000BF00BF00BF00BF94E70000C00C0040CB
:1022900000F4FFBFC00D0040F0B502460D4600201F
:1022A000002407E00126A6402E40002E01D0204643
:1022B00002E0641C102CF5D300BF102C00D1F0BD3F
:1022C0003F4FD61BBA4234D008DC3E4E9619002E42
:1022D0002CD0402E2BD0802E6ED129E0402E02D063
:1022E000802E69D100E000BF0B2800D965E00328EB
:1022F00001D8002106E0042803D3072801D80221D1
:1023000000E004212E4E8036B24200D10831800711
:10231000800F2D4E736803268E401F46B7433B4601
:1023200006468E403343284E736046E000BF00BF30
:1023300000BF234EC03EB24207D0214E803EB24283
:1023400003D01F4E403EB24202D10F2800D934E0E4
:102350001B4EB24202D10B2800D92EE0032801D82F
:1023600000210CE0042803D3072801D8022106E04D
:10237000082803D30B2801D8042100E00621104EC1
:10238000803EB24200D108310D4E403EB24200D1F3
:1023900010310B4EB24200D118318007800F0A4E27
:1023A000336803268E401F46B7433B4606468E40A1
:1023B0003343054E336000E000BF00BF00BF7EE73F
:1023C000C00C004000F4FFBFC00D0040F0B5044653
:1023D0000025002307E001269E400E403546002DD3
:1023E00000D002E05B1C102BF5D300BF102B36D2BF
:1023F0001D46116026680E403046E840012802D193
:102400000126D67101E00026D67166680E40EE40C6
:102410003046012801D1967101E000269671A66828
:102420000E40EE403046012801D1567101E00026F1
:102430005671E6686F00FE40B007800F002802D199
:10244000002616710BE0012802D10126167106E064
:10245000022802D10226167101E003261671F0BD92
:1024600010B501213148FFF781F931493148FFF7B3
:102470002EFB31492F484030FFF729FB2F492D48CB
:102480008030FFF724FBFF2134312A48C030FFF7AA
:102490001EFB172149012A48FFF719FB2949284843
:1024A0004030FFF714FB8C2125488030FFF70FFBED
:1024B00009212548FFF7E0FA012211022048803067
:1024C00000F00DFE012251021D48803000F007FE91
:1024D0000020FFF72BF9002005F054F90020FFF74A
:1024E00001F900211948FFF741F900211748001DA3
:1024F000FFF73CF900211648FFF738F9002113488F
:102500000F30FFF733F90020FFF7B6F80021012064
:102510008006FFF72BF900210448FFF727F9002078
:10252000FFF75CFA0120FFF76BFA10BD070000010E
:102530000F200000000C00400CFB00004060000079
:10254000000D00403FC0000000FC014009000003F6
:1025500004000002F0B502460B46002100240025CD
:1025600000BF2DE001268E4034461E6826403546C9
:10257000A54224D110680646A6433046DE798E4037
:102580003043106050680646A64330469E798E4020
:102590003043506090680646A64330465E798E40D0
:1025A000304390604F000326BE403446D068064654
:1025B000A64330461E794F00BE403043D060491CD0
:1025C0001029CFD3F0BD02460020D3690B40002B69
:1025D00001D0012000E00020704781617047416117
:1025E000704702690A40002A01D0816100E0416120
:1025F000704710B51346826A012B03D114460C4371
:10260000224602E014468C432246826210BD00003E
:1026100070B500250020644948706449087000F0D6
:10262000CBFC634800786349097840186249087018
:10263000084600785F49087000205D4908705E48D0
:102640000078642802DD01205B4908705B4800685F
:1026500059490978884209D25848006858494018B1
:1026600055490978401A5749086006E05348006800
:1026700051490978401A5349086000F0CDFB052004
:1026800049498870122088714F48017B46482330A1
:102690000171090A417101214C4881750021C17500
:1026A0004148233041790279080210431E2807DB94
:1026B0003D4823304179027908021043FF2805DDA7
:1026C0005A2139482330017100214171002557E01A
:1026D00000F072FC0A2006F0F9F86D1C3248807890
:1026E000002804D030488078032800D100BF2E484D
:1026F0008078002803D02C49887904F037F82A48DC
:1027000023304179027908021043002802D0304872
:10271000854235D32FA000F067F800F04DFCC820AB
:1027200006F0D4F81920400106F0D0F8C82006F0D1
:10273000CDF81920400106F0C9F80020274908709B
:102740001A4908700121214881750021C17524486A
:10275000C07C401CC1B22248C174203800780028D7
:1027600005DD1F48807C401CC1B21D4881740021DA
:102770001C48C17201730C482030417200F01CFCEF
:102780000A4800780028A3D100240AE000F014FCD5
:10279000C82006F09BF81920400106F097F8601C4D
:1027A00084B2142CF2DB70BD881D002002060020CC
:1027B0000E0600200F060020100600201406002040
:1027C000EE020000DC0500201C1A0020B31D0020D2
:1027D00050C300004154434C4F53450004060020B1
:1027E000911A0020771D002070B504462046FDF7A1
:1027F00017FDC6B2002505E0207806F087F9641CB5
:10280000681CC5B2B542F7DB012006F05FF870BD69
:1028100070B5002400250120FEF7B0F9FEF762FA3A
:1028200005F03CFD002803D1FEF7ECF9054601E078
:10283000002070BD284605F0ADFC04462046F8E7B0
:1028400038B50020009000240120FEF797F9FEF72C
:1028500049FA05F023FD002803D1FEF7D3F9044619
:1028600001E0002038BD204605F0E6FC009000980D
:10287000F8E70000F0B587B00026FEF7C9F910218F
:102880001F48FFF7ACFE132006F066F9041E30D097
:10289000082161700021A1700A202070204600F0FC
:1028A0004BFA07463846FDF73BFF0190FDF7C4FFA2
:1028B000144A154B03910290FDF752FE05910490C6
:1028C000FDF7E2FF05462846FDF7B6FF0F4A104B1D
:1028D00003910290FDF744FE05910490FDF7D4FFAB
:1028E000064610210648FFF778FE204606F0D8F885
:1028F00000240020FEF742F9304607B0F0BD00008A
:10290000400D0040FCA9F1D24D62503F9A9999992F
:1029100099990540F0B587B00026FEF7A7F9082180
:102920001F48FFF75CFE142006F016F9041E30D095
:10293000082161700021A17005202070204600F060
:10294000FBF907463846FDF7EBFE0190FDF774FFF3
:10295000144A154B03910290FDF702FE0591049075
:10296000FDF792FF05462846FDF766FF0F4A104B1C
:1029700003910290FDF7F4FD05910490FDF784FFAB
:10298000064608210648FFF728FE204606F088F88C
:1029900000240020FEF7F2F8304607B0F0BD00003A
:1029A000400D0040FCA9F1D24D62503F9A9999998F
:1029B0009999094070B5FEF7A5F9132006F0CCF8F7
:1029C000041E0AD0082161700021A170FFF720FFCA
:1029D0000546204606F064F800240020FEF7CEF8F5
:1029E000284670BDF0B585B006460127002523E0D6
:1029F00002A804F045F9684604F042F9002408E012
:102A000002A8005D6946095D884200D003E0601CB1
:102A1000C4B2072CF4DB00BF072C0BD10027072220
:102A200002A93046FDF7C4FB072202A90548FDF7BD
:102A3000BFFB03E0681CC5B2032DD9DB00BF3846DD
:102A400005B0F0BDA00400200EB50722AA49002061
:102A500004F012F8A8480078F0210840002819DB9B
:102A6000A54800780840502814DCA34800780007E7
:102A7000000F00280ADBA04800780007000F092893
:102A800004DC9D4800789D49887006E000209B4941
:102A9000887002E000209949887097484078F021BA
:102AA0000840002819DB944840780840502814DC7E
:102AB000914840780007000F00280ADB8E484078D4
:102AC0000007000F092804DC8B4840788B494870C8
:102AD00006E000208949487002E0002087494870DC
:102AE00085488078F021084000110A214843824936
:102AF00089780907090F4018182823DA7E4880785A
:102B0000F0210840002819DB7B4880780840202805
:102B100014DC794880780007000F00280ADB76482B
:102B200080780007000F092804DC73488078734917
:102B300008700AE000207149087006E000206F4923
:102B4000087002E000206D4908706B48C0786B493E
:102B5000487169480079F021084000110A21484372
:102B6000654909790907090F4018202831DA6248B8
:102B70000079F021084000110A2148435E49097993
:102B80000907090F4018002823DD5B480079F02170
:102B90000840002819DB584800790840302814DC28
:102BA000554800790007000F00280ADB52480079D9
:102BB0000007000F092804DC4F4800794F490871CD
:102BC0000AE001204D49087106E001204B490871D7
:102BD00002E001204949087147484079F021084046
:102BE00000110A214843444949790907090F40184F
:102BF0000D2831DA40484079F021084000110A21BF
:102C000048433D4949790907090F4018002823DD49
:102C100039484079F0210840002819DB36484079CE
:102C20000840102814DC344840790007000F0028C1
:102C30000ADB314840790007000F092804DC2E48E0
:102C400040792E49C8700AE012202C49C87006E06D
:102C500012202A49C87002E012202849C87026486C
:102C60008079F021084000110A21484322498979DE
:102C70000907090F4018642826DA1F488079F021D7
:102C8000084000281CDB1C4880790840902817DC8D
:102C9000194880790007000F00280DDB164880795D
:102CA0000007000F092807DC134880790121490338
:102CB00040181249C8800AE011481049C88006E04F
:102CC0000F480E49C88002E00D480C49C8806420B6
:102CD00005F0FCFD0948807808494978074A1278D0
:102CE00000920191029005480379C278C18805A03D
:102CF00004F09CFD0EBD0000C62000201A06002036
:102D00001520000045585445524E414C2052544322
:102D10002054494D45203D2025582D253032582D31
:102D2000253032582D253032582D253032582D255A
:102D3000303258200D0A0000FEB5044600200090F5
:102D4000002509E0FFF77CFD0746AA00E01C1118EA
:102D50003846FDF776FA6D1CA178627808021043B8
:102D6000A842EFD800252EE06E1C25E0B200E11C41
:102D70005018FDF75CFA0746AA00E11C5018FDF751
:102D800056FA874217D2B200E11C5018FDF74FFAED
:102D90000190AA00E11C5018FDF749FA0746B2005D
:102DA000E01C11183846FDF74CFAAA00E01C111877
:102DB0000198FDF746FA761CA17862780802104364
:102DC000B042D3D86D1CA178627808021043A842A3
:102DD000CAD8012002900BE002998A00E11C501829
:102DE000FDF725FA0099401800900298401C0290C7
:102DF000A178627808021043401E02998842EBD8FD
:102E0000A278637810021843811E0098FDF776F9C6
:102E100000900098FEBD000010B588B020216846E3
:102E2000FDF7DFF91A21684601704170002405E0C2
:102E30000021A01C6A461154601CC4B2082CF7DBA8
:102E40002720214908706C20487051208870692023
:102E5000C870AA21684681732621C173002407E047
:102E60001948015D20460A306A461154601CC4B2FC
:102E7000042CF5DBFF216846017400214174002415
:102E800006E00021204612306A461154601CC4B28C
:102E9000072CF6DB002069464876002409E06846E6
:102EA000407E6946095D4018C1B268464176601CA3
:102EB000C4B2192CF3DB1620694688761E2203481B
:102EC00004F008FC08B010BDFA05002000680140BD
:102ED00010B50F488078012818D10EA004F0A6FC88
:102EE000002406E00E48015D0EA004F09FFC601C6B
:102EF00084B207494878097800020843A042F1DC0F
:102F00000AA004F093FC00200149887010BD000065
:102F1000441600204D43553C2D477273200000009D
:102F20004412002030782530327820000D0A00004D
:102F300070B500260320FEF735FF05461C48854284
:102F400016D0022005F0C2FC0CE00320FEF72AFF99
:102F50000546022005F0BAFC3046711C8EB264288A
:102F600000DD04E00320FEF71DFFA842EDD101E0E3
:102F7000012070BD0E48281A84B2002C15D00D48CF
:102F800004800320FEF730FF00210320FEF7E4FE5B
:102F900007490320FEF70EFF01210320FEF7DCFEA8
:102FA0000120044988700020E3E70120E1E70000E8
:102FB000441200204416002001480249086070476E
:102FC0005A5A34120014014010B501210448FEF78A
:102FD000CDFB062003494860FFF7EEFF10BD00005F
:102FE000050000010014014010B501210648FEF75C
:102FF000BDFB00220821054803F036FC0022042115
:10300000024803F031FC10BD07000001C00C004075
:103010001CB5002000900120694608716846FEF743
:1030200039FC0120FEF7FEFA1CBD00000A2005490C
:1030300008600548008CC0B20449C86105200149F8
:103040000860704700E0014000FBFF1F00F80140EE
:103050001FB5002401211948FEF788FB02211848FA
:10306000FEF767F804211648FEF763F80120FEF723
:1030700085FC07200002FEF793FC052005F026FCE6
:103080000120FEF7ADFA05E019200002844200D3CA
:1030900004E0641CFEF7B8FA0028F5D000BF012058
:1030A0000090002001900290012069460873684654
:1030B000FEF754FC034805F0E5FB1FBD07000001C7
:1030C000400D0040001BB70010B50020FEF722FFA6
:1030D000FFF79EFFFFF7AAFFFFF7BAFF10BD7FB50E
:1030E00006460D4614466A4629463046FFF76EF9F5
:1030F0000098A84217D16846C079012813D16846C4
:10310000407901280FD1002C03D16846807900282E
:1031100009D1012C03D168468079012803D1684682
:103120000079002814D0029501216846C1734173CB
:10313000002C03D100206946887302E00120694613
:10314000887300206946087302A93046FFF702FA27
:103150007FBD0000F8B505460E4600240027FEF7A7
:1031600097F9002802D10120FEF79EF9002426E0FD
:103170000120A04007462846384000281ED0002ED7
:1031800007D1144840680121A14088431149486093
:1031900006E0104840680121A14008430D494860FD
:1031A0000C48816862000320904081430948816097
:1031B00000680121A140084306490860641C042CF2
:1031C000D6D3FEF765F9012802D10020FEF76CF98D
:1031D000F8BD000000FC014010B500240A20FDF7F6
:1031E0000BFE09240AE000F071FA00F0BBFA204659
:1031F000FDF702FE00F00CF8601EC4B2002CF2DCF9
:1032000000F064FA00F0AEFA0020FDF7F5FD10BD05
:1032100030B589B0002008904FE208988000FE4940
:103220000968085C079008988000FB490968401805
:103230004078069008988100F74800680818807860
:10324000059008988000F44909684018C0780490F7
:10325000079805F0ADFF0446079805F0A9FF039015
:1032600005F0A6FF4440079805F0A2FF029005F084
:103270009FFF039005F09CFF4440079805F098FFDE
:10328000019005F095FF029005F092FF039005F084
:103290008FFF069805F08CFF05460698454005F01F
:1032A00087FF039005F084FF069805F081FF0290E8
:1032B00005F07EFF039005F07BFF4540069805F082
:1032C00077FF019005F074FF029005F071FF039005
:1032D00005F06EFF6C40059805F06AFF05980546FD
:1032E00005F066FF039005F063FF4540059805F083
:1032F0005FFF029005F05CFF039005F059FF454029
:10330000059805F055FF019005F052FF029005F079
:103310004FFF039005F04CFF6C40049805F048FF08
:103320000498054605F044FF039005F041FF04981A
:1033300005F03EFF029005F03BFF039005F038FFDB
:103340004540049805F034FF019005F031FF0290EC
:1033500005F02EFF039005F02BFF6C4008988000CD
:10336000AD4909680C54079805F022FF07980446F8
:1033700005F01EFF039005F01BFF079805F018FFEE
:10338000029005F015FF039005F012FF44400798E6
:1033900005F00EFF019005F00BFF029005F008FF0D
:1033A000039005F005FF069805F002FF0546069814
:1033B00005F0FEFE039005F0FBFE4540069805F083
:1033C000F7FE029005F0F4FE039005F0F1FE454093
:1033D000069805F0EDFE019005F0EAFE029005F07A
:1033E000E7FE039005F0E4FE6C40059805F0E0FE72
:1033F00005460598454005F0DBFE039005F0D8FE34
:10340000059805F0D5FE029005F0D2FE039005F078
:10341000CFFE4540059805F0CBFE019005F0C8FEB3
:10342000029005F0C5FE039005F0C2FE6C400498C2
:1034300005F0BEFE0498054605F0BAFE039005F0BF
:10344000B7FE4540049805F0B3FE029005F0B0FECB
:10345000039005F0ADFE4540049805F0A9FE0190EB
:1034600005F0A6FE029005F0A3FE039005F0A0FE75
:103470006C400898800068490968401844700798B3
:1034800005F096FE0798044605F092FE039005F0BD
:103490008FFE4440079805F08BFE029005F088FEF1
:1034A000039005F085FE4440079805F081FE0190E9
:1034B00005F07EFE029005F07BFE039005F078FE9D
:1034C000069805F075FE0698054605F071FE039016
:1034D00005F06EFE069805F06BFE029005F068FEA2
:1034E000039005F065FE4540069805F061FE0190E9
:1034F00005F05EFE029005F05BFE039005F058FEBD
:103500006C40059805F054FE0546059805F050FE00
:10351000039005F04DFE4540059805F049FE0290E8
:1035200005F046FE039005F043FE4540059805F082
:103530003FFE019005F03CFE029005F039FE03903D
:1035400005F036FE6C40049805F032FE05460498FE
:10355000454005F02DFE039005F02AFE049805F085
:1035600027FE029005F024FE039005F021FE454061
:10357000049805F01DFE019005F01AFE029005F07A
:1035800017FE039005F014FE6C4008988000224A54
:10359000126880188470079805F00AFE04460798A0
:1035A000444005F005FE039005F002FE079805F083
:1035B000FFFD029005F0FCFD039005F0F9FD44408D
:1035C000079805F0F5FD019005F0F2FD029005F079
:1035D000EFFD039005F0ECFD069805F0E9FD069877
:1035E000054605F0E5FD039005F0E2FD454006982F
:1035F00005F0DEFD029005F0DBFD039005F0D8FD3F
:103600004540069805F0D4FD019005F0D1FD0290EB
:1036100005F0CEFD039001E03404002005F0C8FD64
:103620006C40059805F0C4FD0598054605F0C0FD01
:10363000039005F0BDFD059805F0BAFD029005F078
:10364000B7FD039005F0B4FD4540059805F0B0FDC9
:10365000019005F0ADFD029005F0AAFD039005F084
:10366000A7FD6C40049805F0A3FD0546049805F0FD
:103670009FFD039005F09CFD4540049805F098FDE2
:10368000029005F095FD039005F092FD45400498E9
:1036900005F08EFD019005F08BFD029005F088FD90
:1036A000039005F085FD6C4008988000064A12687A
:1036B0008018C4700898401C08900898042800DA04
:1036C000ABE509B030BD000034040020244909688E
:1036D000487B234909684A7A214909684A73204985
:1036E00009684A791E4909684A721D4909684A7879
:1036F0001B4909684A711A490968487018490968DC
:10370000887817490968897A154A126891701449AE
:1037100009688872124909688879114909688A7BA1
:103720000F4909688A710E49096888730C4909684C
:10373000C8780B490968C979094A1268D1700849E3
:103740000968CA7A06490968CA7105490968CA7BC5
:1037500003490968CA7202490968C87370470000C2
:103760003404002070B5002413E000250DE0A9000A
:10377000094A12688918085D05F0BCF9A900064AD3
:10378000126889180855681CC5B2042DEFDB601C4F
:10379000C4B2042CE9DB70BD34040020F8B5002469
:1037A0001FE0A00043490968095CA000424A115487
:1037B000A000401C3F490968095CA000401C11544E
:1037C000A000801C3B490968095CA000801C1154C2
:1037D000A000C01C37490968095CA000C01C115436
:1037E000641C042CDDD362E0002507E0601E80002D
:1037F00040193149085C694648556D1C042DF5D3C4
:10380000A007800F002825D168460678417801700E
:1038100081784170C1788170C6706946087805F07A
:103820006FF969460870487805F06AF9694648708A
:10383000887805F065F969468870C87805F060F900
:103840006946C8700878A1081C4A515C484069461E
:10385000087000E000BF201F80001749085C69461F
:1038600009784840A100144A5054201F8000401C91
:103870001146095C684640784840A100491C5054F4
:10388000201F8000801C1146095C684680784840F3
:10389000A100891C5054201F8000C01C1146085CE8
:1038A0006946C9784840A100C91C5054641C2C2C9E
:1038B0009AD3F8BD38040020E8170020C293000016
:1038C00010B5FF20153002F001FCFF20163002F089
:1038D000FDFBFF200F3002F0F9FBFF20103002F05B
:1038E000F5FBFF20183002F0F1FBFF20173002F04B
:1038F000EDFBFF200E3002F0E9FBFF200D3002F05F
:10390000E5FB052002F0E2FB062002F0DFFB0720CA
:1039100002F0DCFB042002F0D9FB572002F0D6FBBA
:103920003F2002F0D3FB472002F0D0FB462002F0FC
:10393000CDFB452002F0CAFB4D2002F0C7FB4E2014
:1039400002F0C4FB4F2002F0C1FB502002F0BEFB8E
:10395000492002F0BBFB4A2002F0B8FB402002F0F5
:10396000B5FB422002F0B2FB4B2002F0AFFB482037
:1039700002F0ACFB412002F0A9FB3C2002F0A6FBC8
:10398000442002F0A3FB4C2002F0A0FB432002F0F5
:103990009DFB022002F09AFB032002F097FB01201E
:1039A00002F094FB002002F091FBFF20143002F0A3
:1039B0008DFBFF20133002F089FBFF20123002F054
:1039C00085FBFF200B3002F081FBFF200C3002F062
:1039D0007DFBFF20053002F079FBFF20113002F063
:1039E00075FBFF200A3002F071FBFF20093002F066
:1039F0006DFB8B2002F06AFB822002F067FB8320C4
:103A000002F064FB8C2002F061FB812002F05EFB7F
:103A1000802002F05BFB8E2002F058FB872002F032
:103A200055FB862002F052FB852002F04FFB8420DC
:103A300002F04CFB132002F049FB182002F046FB79
:103A4000FF20033002F042FBFF20013002F03EFB7A
:103A5000F22002F03BFBF02002F038FBE32002F002
:103A600035FBE02002F032FBD32002F02FFBC82010
:103A700002F02CFBBA2002F029FBB82002F026FB52
:103A8000AA2002F023FBA82002F020FB9B2002F0DA
:103A90001DFB982002F01AFBF52002F017FBF7201F
:103AA00002F014FBE52002F011FBE72002F00EFB10
:103AB000D42002F00BFBD72002F008FBC42002F058
:103AC00005FBBF2002F002FBAD2002F0FFFAAF20A1
:103AD00002F0FCFA9D2002F0F9FA9F2002F0F6FABB
:103AE0000821012000F079F80821022000F075F883
:103AF0000821032000F071F80821042000F06DF87F
:103B00000821052000F069F80821062000F065F87A
:103B10000821072000F061F80821084600F05DF850
:103B20000821092000F059F808210A2000F055F872
:103B300008210B2000F051F808210C2000F04DF86E
:103B400008210D2000F049F808210E2000F045F86A
:103B500008210F2000F041F80821102000F03DF866
:103B60000821112000F039F80821122000F035F862
:103B70000821132000F031F80821142000F02DF85E
:103B8000014802F0BFFA10BD9620002030B5014672
:103B9000C3175B0F5B18DB10094CE35C0246C417CC
:103BA000640FA418E410E400051B0124AC40A343F7
:103BB000C417640F6418E410014D2B5530BD00008C
:103BC0009620002000B58DB0302101A8FCF709FB3C
:103BD00001A802F097FA0DB000BD70B505460C467D
:103BE000152D01D302F06FFA6B007B449B885B00BC
:103BF0009F4469121400FC00E401CC02B4039C044D
:103C000084058106690751083909210A090BF10B5E
:103C1000F90CE10DC90EB10F99108111230003F0C9
:103C200040FE0A061C32485E748AA0B6CCE20F2021
:103C300002F04CFA172002F049FA152002F046FA79
:103C40000C2002F043FA0D2002F040FA0E2002F0A0
:103C50003DFA1620FFF79AFFC6E00F20FFF796FF08
:103C6000172002F033FA152002F030FA0C20FFF78B
:103C70008DFF0D20FFF78AFF0E20FFF787FF16202C
:103C8000FFF784FFB0E00F2002F020FA172002F0C7
:103C90001DFA1520FFF77AFF0C2002F017FA0D200D
:103CA00002F014FA0E20FFF771FF162002F00EFA50
:103CB0009AE00F2002F00AFA172002F007FA152006
:103CC00002F004FA0C2002F001FA0D20FFF75EFF6B
:103CD0000E20FFF75BFF162002F0F8F984E00F20BA
:103CE000FFF754FF172002F0F1F9152002F0EEF96A
:103CF0000C20FFF74BFF0D20FFF748FF0E2002F0CE
:103D0000E5F9162002F0E2F96EE00F2002F0DEF98C
:103D10001720FFF73BFF152002F0D8F90C2002F026
:103D2000D5F90D20FFF732FF0E2002F0CFF9162053
:103D300002F0CCF958E00F2002F0C8F91720FFF785
:103D400025FF152002F0C2F90C2002F0BFF90D206A
:103D500002F0BCF90E2002F0B9F9162002F0B6F913
:103D600042E00F2002F0B2F9172002F0AFF915205F
:103D700002F0ACF90C20FFF709FF0D20FFF706FF5A
:103D80000E20FFF703FF1620FFF700FF2CE00F20A7
:103D900002F09CF9172002F099F9152002F096F92B
:103DA0000C2002F093F90D2002F090F90E2002F0A1
:103DB0008DF9162002F08AF916E00F2002F086F93C
:103DC000172002F083F9152002F080F90C2002F090
:103DD0007DF90D20FFF7DAFE0E2002F077F91620AC
:103DE00002F074F900E000BF00BFFBE6230003F01F
:103DF00058FD0A061C32485E748AA0B6CCE21F2029
:103E000002F064F93E2002F061F93D2002F05EF913
:103E10001C2002F05BF9142002F058F91E2002F079
:103E200055F91D20FFF7B2FEC6E01F20FFF7AEFEDA
:103E30003E2002F04BF93D2002F048F91C20FFF72C
:103E4000A5FE1420FFF7A2FE1E20FFF79FFE1D20F7
:103E5000FFF79CFEB0E01F2002F038F93E2002F090
:103E600035F93D20FFF792FE1C2002F02FF91420B7
:103E700002F02CF91E20FFF789FE1D2002F026F922
:103E80009AE01F2002F022F93E2002F01FF93D20A7
:103E900002F01CF91C2002F019F91420FFF776FE3D
:103EA0001E20FFF773FE1D2002F010F984E01F2092
:103EB000FFF76CFE3E2002F009F93D2002F006F902
:103EC0001C20FFF763FE1420FFF760FE1E2002F0A7
:103ED000FDF81D2002F0FAF86EE01F2002F0F6F85F
:103EE0003E20FFF753FE3D2002F0F0F81C2002F0C8
:103EF000EDF81420FFF74AFE1E2002F0E7F81D201F
:103F000002F0E4F858E01F2002F0E0F83E20FFF74E
:103F10003DFE3D2002F0DAF81C2002F0D7F8142014
:103F200002F0D4F81E2002F0D1F81D2002F0CEF8E5
:103F300042E01F2002F0CAF83E2002F0C7F83D2000
:103F400002F0C4F81C20FFF721FE1420FFF71EFE2C
:103F50001E20FFF71BFE1D20FFF718FE2CE01F2080
:103F600002F0B4F83E2002F0B1F83D2002F0AEF8C5
:103F70001C2002F0ABF8142002F0A8F81E2002F07A
:103F8000A5F81D2002F0A2F816E01F2002F09EF80E
:103F90003E2002F09BF83D2002F098F81C2002F031
:103FA00095F81420FFF7F2FD1E2002F08FF81D2077
:103FB00002F08CF800E000BF00BF13E6230003F01E
:103FC00070FC0A061C32485E748AA0B6CCE25F2000
:103FD00002F07CF85E2002F079F85D2002F076F8BD
:103FE0005C2002F073F8542002F070F8562002F0C2
:103FF0006DF85520FFF7CAFDC6E05F20FFF7C6FD4C
:104000005E2002F063F85D2002F060F85C20FFF7AC
:10401000BDFD5420FFF7BAFD5620FFF7B7FD552030
:10402000FFF7B4FDB0E05F2002F050F85E2002F030
:104030004DF85D20FFF7AAFD5C2002F047F8542000
:1040400002F044F85620FFF7A1FD552002F03EF89B
:104050009AE05F2002F03AF85E2002F037F85D2027
:1040600002F034F85C2002F031F85420FFF78EFDA6
:104070005620FFF78BFD552002F028F884E05F20E2
:10408000FFF784FD5E2002F021F85D2002F01EF8AB
:104090005C20FFF77BFD5420FFF778FD562002F0EF
:1040A00015F8552002F012F86EE05F2002F00EF8CD
:1040B0005E20FFF76BFD5D2002F008F85C2002F047
:1040C00005F85420FFF762FD562001F0FFFF552050
:1040D00001F0FCFF58E05F2001F0F8FF5E20FFF7E1
:1040E00055FD5D2001F0F2FF5C2001F0EFFF542050
:1040F00001F0ECFF562001F0E9FF552001F0E6FF4A
:1041000042E05F2001F0E2FF5E2001F0DFFF5D2072
:1041100001F0DCFF5C20FFF739FD5420FFF736FD8E
:104120005620FFF733FD5520FFF730FD2CE05F20D0
:1041300001F0CCFF5E2001F0C9FF5D2001F0C6FF59
:104140005C2001F0C3FF542001F0C0FF562001F0B5
:10415000BDFF552001F0BAFF16E05F2001F0B6FF69
:104160005E2001F0B3FF5D2001F0B0FF5C2001F0A4
:10417000ADFF5420FFF70AFD562001F0A7FF5520A0
:1041800001F0A4FF00E000BF00BF2BE5230003F017
:1041900088FB0A061C32485E748AA0B6CCE258201E
:1041A00001F094FF512001F091FF532001F08EFFA8
:1041B0005B2001F08BFF5A2001F088FF592001F0AD
:1041C00085FF5220FFF7E2FCC6E05820FFF7DEFC37
:1041D000512001F07BFF532001F078FF5B20FFF7B7
:1041E000D5FC5A20FFF7D2FC5920FFF7CFFC522014
:1041F000FFF7CCFCB0E0582001F068FF512001F03F
:1042000065FF5320FFF7C2FC5B2001F05FFF5A20DF
:1042100001F05CFF5920FFF7B9FC522001F056FF76
:104220009AE0582001F052FF512001F04FFF532037
:1042300001F04CFF5B2001F049FF5A20FFF7A6FC7C
:104240005920FFF7A3FC522001F040FF84E05820E2
:10425000FFF79CFC512001F039FF532001F036FF9D
:104260005B20FFF793FC5A20FFF790FC592001F0E8
:104270002DFF522001F02AFF6EE0582001F026FFAA
:104280005120FFF783FC532001F020FF5B2001F059
:104290001DFF5A20FFF77AFC592001F017FF52202A
:1042A00001F014FF58E0582001F010FF5120FFF7F3
:1042B0006DFC532001F00AFF5B2001F007FF5A203C
:1042C00001F004FF592001F001FF522001F0FEFE31
:1042D00042E0582001F0FAFE512001F0F7FE532091
:1042E00001F0F4FE5B20FFF751FC5A20FFF74EFC73
:1042F0005920FFF74BFC5220FFF748FC2CE05820D8
:1043000001F0E4FE512001F0E1FE532001F0DEFE59
:104310005B2001F0DBFE5A2001F0D8FE592001F0AD
:10432000D5FE522001F0D2FE16E0582001F0CEFE5C
:10433000512001F0CBFE532001F0C8FE5B2001F0BC
:10434000C5FE5A20FFF722FC592001F0BFFE522083
:1043500001F0BCFE00E000BF00BF43E4230003F017
:10436000A0FA0A061C32485E748AA0B6CCE20B2082
:1043700001F0ACFE122001F0A9FE102001F0A6FE13
:10438000082001F0A3FE092001F0A0FE0A2001F0A0
:104390009DFE1120FFF7FAFBC6E00B20FFF7F6FBAE
:1043A000122001F093FE102001F090FE0820FFF78C
:1043B000EDFB0920FFF7EAFB0A20FFF7E7FB1120DE
:1043C000FFF7E4FBB0E00B2001F080FE122001F0CB
:1043D0007DFE1020FFF7DAFB082001F077FE0920B0
:1043E00001F074FE0A20FFF7D1FB112001F06EFEF0
:1043F0009AE00B2001F06AFE122001F067FE102007
:1044000001F064FE082001F061FE0920FFF7BEFB09
:104410000A20FFF7BBFB112001F058FE84E00B20BF
:10442000FFF7B4FB122001F051FE102001F04EFE08
:104430000820FFF7ABFB0920FFF7A8FB0A2001F0DB
:1044400045FE112001F042FE6EE00B2001F03EFE21
:104450001220FFF79BFB102001F038FE082001F02E
:1044600035FE0920FFF792FB0A2001F02FFE1120F4
:1044700001F02CFE58E00B2001F028FE1220FFF77F
:1044800085FB102001F022FE082001F01FFE09200C
:1044900001F01CFE0A2001F019FE112001F016FEA9
:1044A00042E00B2001F012FE122001F00FFE10205E
:1044B00001F00CFE0820FFF769FB0920FFF766FBFF
:1044C0000A20FFF763FB1120FFF760FB2CE00B20B5
:1044D00001F0FCFD122001F0F9FD102001F0F6FDC5
:1044E000082001F0F3FD092001F0F0FD0A2001F0A1
:1044F000EDFD112001F0EAFD16E00B2001F0E6FDD4
:10450000122001F0E3FD102001F0E0FD082001F091
:10451000DDFD0920FFF73AFB0A2001F0D7FD11204D
:1045200001F0D4FD00E000BF00BF5EE4230003F013
:10453000B8F90A061C32485E748AA0B6CCE23B2069
:1045400001F0C4FD3A2001F0C1FD392001F0BEFDAB
:10455000382001F0BBFD192001F0B8FD1B2001F04F
:10456000B5FD1A20FFF712FBC6E03B20FFF70EFB5C
:104570003A2001F0ABFD392001F0A8FD3820FFF70B
:1045800005FB1920FFF702FB1B20FFF7FFFA1A209B
:10459000FFF7FCFAB0E03B2001F098FD3A2001F073
:1045A00095FD3920FFF7F2FA382001F08FFD192030
:1045B00001F08CFD1B20FFF7E9FA1A2001F086FDBF
:1045C0009AE03B2001F082FD3A2001F07FFD392086
:1045D00001F07CFD382001F079FD1920FFF7D6FAB3
:1045E0001B20FFF7D3FA1A2001F070FD84E03B2076
:1045F000FFF7CCFA3A2001F069FD392001F066FDA1
:104600003820FFF7C3FA1920FFF7C0FA1B2001F08A
:104610005DFD1A2001F05AFD6EE03B2001F056FDD1
:104620003A20FFF7B3FA392001F050FD382001F0AD
:104630004DFD1920FFF7AAFA1B2001F047FD1A20B3
:1046400001F044FD58E03B2001F040FD3A20FFF727
:104650009DFA392001F03AFD382001F037FD19208C
:1046600001F034FD1B2001F031FD1A2001F02EFD78
:1046700042E03B2001F02AFD3A2001F027FD3920DD
:1046800001F024FD3820FFF781FA1920FFF77EFAA8
:104690001B20FFF77BFA1A20FFF778FA2CE03B206B
:1046A00001F014FD3A2001F011FD392001F00EFD5A
:1046B000382001F00BFD192001F008FD1B2001F04E
:1046C00005FD1A2001F002FD16E03B2001F0FEFC82
:1046D0003A2001F0FBFC392001F0F8FC382001F011
:1046E000F5FC1920FFF752FA1B2001F0EFFC1A200D
:1046F00001F0ECFC00E000BF00BF5EE4230003F02B
:10470000D0F80A061E364E667E96AEC6DEF7FB2051
:1047100001F0DCFCF32001F0D9FCF92001F0D6FC1B
:10472000F82001F0D3FCFF20023001F0CFFCFF2085
:10473000043001F0CBFCFA20FFF728FAD9E0FB2087
:10474000FFF724FAF32001F0C1FCF92001F0BEFCD0
:10475000F820FFF71BFAFF200230FFF717FAFF20BF
:104760000430FFF713FAFA20FFF710FAC1E0FB203C
:1047700001F0ACFCF32001F0A9FCF920FFF706FAE8
:10478000F82001F0A3FCFF20023001F09FFCFF2085
:104790000430FFF7FBF9FA2001F098FCA9E0FB20B8
:1047A00001F094FCF32001F091FCF92001F08EFC63
:1047B000F82001F08BFCFF200230FFF7E7F9FF2023
:1047C0000430FFF7E3F9FA2001F080FC91E0FB20D0
:1047D000FFF7DCF9F32001F079FCF92001F076FC19
:1047E000F820FFF7D3F9FF200230FFF7CFF9FF20C1
:1047F000043001F06BFCFA2001F068FC79E0FB204A
:1048000001F064FCF320FFF7C1F9F92001F05EFC30
:10481000F82001F05BFCFF200230FFF7B7F9FF2022
:10482000043001F053FCFA2001F050FC61E0FB2061
:1048300001F04CFCF320FFF7A9F9F92001F046FC48
:10484000F82001F043FCFF20023001F03FFCFF2084
:10485000043001F03BFCFA2001F038FC49E0FB2079
:1048600001F034FCF32001F031FCF92001F02EFCC2
:10487000F820FFF78BF9FF200230FFF787F9FF20C0
:104880000430FFF783F9FA20FFF780F931E0FB20CD
:1048900001F01CFCF32001F019FCF92001F016FCDA
:1048A000F82001F013FCFF20023001F00FFCFF2084
:1048B000043001F00BFCFA2001F008FC19E0FB20A9
:1048C00001F004FCF32001F001FCF92001F0FEFBF3
:1048D000F82001F0FBFBFF200230FFF757F9FF2023
:1048E000043001F0F3FBFA2001F0F0FB01E0FFE7F8
:1048F00000BF00BF49E4230002F0D3FF0A061C32C8
:10490000485E748AA0B6CCE2EB2001F0DFFBE22027
:1049100001F0DCFBE12001F0D9FBE82001F0D6FB3F
:10492000F12001F0D3FBEA2001F0D0FBE920FFF7F2
:104930002DF9C6E0EB20FFF729F9E22001F0C6FBD4
:10494000E12001F0C3FBE820FFF720F9F120FFF799
:104950001DF9EA20FFF71AF9E920FFF717F9B0E08F
:10496000EB2001F0B3FBE22001F0B0FBE120FFF708
:104970000DF9E82001F0AAFBF12001F0A7FBEA20E5
:10498000FFF704F9E92001F0A1FB9AE0EB2001F028
:104990009DFBE22001F09AFBE12001F097FBE8206B
:1049A00001F094FBF120FFF7F1F8EA20FFF7EEF8B1
:1049B000E92001F08BFB84E0EB20FFF7E7F8E22031
:1049C00001F084FBE12001F081FBE820FFF7DEF835
:1049D000F120FFF7DBF8EA2001F078FBE92001F095
:1049E00075FB6EE0EB2001F071FBE220FFF7CEF8E3
:1049F000E12001F06BFBE82001F068FBF120FFF7FC
:104A0000C5F8EA2001F062FBE92001F05FFB58E005
:104A1000EB2001F05BFBE220FFF7B8F8E12001F0AA
:104A200055FBE82001F052FBF12001F04FFBEA209A
:104A300001F04CFBE92001F049FB42E0EB2001F0E2
:104A400045FBE22001F042FBE12001F03FFBE820C2
:104A5000FFF79CF8F120FFF799F8EA20FFF796F8A6
:104A6000E920FFF793F82CE0EB2001F02FFBE22088
:104A700001F02CFBE12001F029FBE82001F026FBEE
:104A8000F12001F023FBEA2001F020FBE92001F0F6
:104A90001DFB16E0EB2001F019FBE22001F016FBF4
:104AA000E12001F013FBE82001F010FBF120FFF7FB
:104AB0006DF8EA2001F00AFBE92001F007FB00E0B5
:104AC00000BF00BF49E4230002F0EBFE0A061C32DF
:104AD000485E748AA0B6CCE2DB2001F0F7FAD2205F
:104AE00001F0F4FAD02001F0F1FAD82001F0EEFA4A
:104AF000D92001F0EBFADA2001F0E8FAD120FFF733
:104B000045F8C6E0DB20FFF741F8D22001F0DEFADD
:104B1000D02001F0DBFAD820FFF738F8D920FFF7D2
:104B200035F8DA20FFF732F8D120FFF72FF8B0E0A0
:104B3000DB2001F0CBFAD22001F0C8FAD020FFF739
:104B400025F8D82001F0C2FAD92001F0BFFADA2006
:104B5000FFF71CF8D12001F0B9FA9AE0DB2001F050
:104B6000B5FAD22001F0B2FAD02001F0AFFAD82085
:104B700001F0ACFAD920FFF709F8DA20FFF706F8C0
:104B8000D12001F0A3FA84E0DB20FEF7FFFFD22062
:104B900001F09CFAD02001F099FAD820FEF7F6FF38
:104BA000D920FEF7F3FFDA2001F090FAD12001F0CE
:104BB0008DFA6EE0DB2001F089FAD220FEF7E6FFE5
:104BC000D02001F083FAD82001F080FAD920FEF736
:104BD000DDFFDA2001F07AFAD12001F077FA58E00F
:104BE000DB2001F073FAD220FEF7D0FFD02001F0D5
:104BF0006DFAD82001F06AFAD92001F067FADA20BC
:104C000001F064FAD12001F061FA42E0DB2001F00A
:104C10005DFAD22001F05AFAD02001F057FAD820DC
:104C2000FEF7B4FFD920FEF7B1FFDA20FEF7AEFFA2
:104C3000D120FEF7ABFF2CE0DB2001F047FAD220B9
:104C400001F044FAD02001F041FAD82001F03EFAF8
:104C5000D92001F03BFADA2001F038FAD12001F036
:104C600035FA16E0DB2001F031FAD22001F02EFAFD
:104C7000D02001F02BFAD82001F028FAD920FEF735
:104C800085FFDA2001F022FAD12001F01FFA00E0BE
:104C900000BF00BF49E4230002F003FE0A061C32F5
:104CA000485E748AA0B6CCE2C32001F00FFAC2209D
:104CB00001F00CFAC12001F009FAC02001F006FA57
:104CC000C92001F003FACB2001F000FACA20FEF758
:104CD0005DFFC6E0C320FEF759FFC22001F0F6F9E0
:104CE000C12001F0F3F9C020FEF750FFC920FEF704
:104CF0004DFFCB20FEF74AFFCA20FEF747FFB0E08A
:104D0000C32001F0E3F9C22001F0E0F9C120FEF771
:104D10003DFFC02001F0DAF9C92001F0D7F9CB201E
:104D2000FEF734FFCA2001F0D1F99AE0C32001F068
:104D3000CDF9C22001F0CAF9C12001F0C7F9C020A5
:104D400001F0C4F9C920FEF721FFCB20FEF71EFFBA
:104D5000CA2001F0BBF984E0C320FEF717FFC22090
:104D600001F0B4F9C12001F0B1F9C020FEF70EFF47
:104D7000C920FEF70BFFCB2001F0A8F9CA2001F0F3
:104D8000A5F96EE0C32001F0A1F9C220FEF7FEFEF6
:104D9000C12001F09BF9C02001F098F9C920FEF76D
:104DA000F5FECB2001F092F9CA2001F08FF958E00E
:104DB000C32001F08BF9C220FEF7E8FEC12001F00C
:104DC00085F9C02001F082F9C92001F07FF9CB20DC
:104DD00001F07CF9CA2001F079F942E0C32001F02A
:104DE00075F9C22001F072F9C12001F06FF9C020FD
:104DF000FEF7CCFEC920FEF7C9FECB20FEF7C6FEAB
:104E0000CA20FEF7C3FE2CE0C32001F05FF9C220E8
:104E100001F05CF9C12001F059F9C02001F056F908
:104E2000C92001F053F9CB2001F050F9CA2001F05C
:104E30004DF916E0C32001F049F9C22001F046F90E
:104E4000C12001F043F9C02001F040F9C920FEF76C
:104E50009DFECB2001F03AF9CA2001F037F900E0BD
:104E600000BF00BF49E4230002F01BFD0A061C320C
:104E7000485E748AA0B6CCE2B32001F027F9AB20DB
:104E800001F024F9B12001F021F9B02001F01EF960
:104E9000B92001F01BF9BB2001F018F9B220FEF790
:104EA00075FEC6E0B320FEF771FEAB2001F00EF9EF
:104EB000B12001F00BF9B020FEF768FEB920FEF733
:104EC00065FEBB20FEF762FEB220FEF75FFEB0E09B
:104ED000B32001F0FBF8AB2001F0F8F8B120FEF7A9
:104EE00055FEB02001F0F2F8B92001F0EFF8BB2038
:104EF000FEF74CFEB22001F0E9F89AE0B32001F091
:104F0000E5F8AB2001F0E2F8B12001F0DFF8B020C5
:104F100001F0DCF8B920FEF739FEBB20FEF736FEC3
:104F2000B22001F0D3F884E0B320FEF72FFEAB20CF
:104F300001F0CCF8B12001F0C9F8B020FEF726FE50
:104F4000B920FEF723FEBB2001F0C0F8B22001F02B
:104F5000BDF86EE0B32001F0B9F8AB20FEF716FE05
:104F6000B12001F0B3F8B02001F0B0F8B920FEF79D
:104F70000DFEBB2001F0AAF8B22001F0A7F858E01E
:104F8000B32001F0A3F8AB20FEF700FEB12001F042
:104F90009DF8B02001F09AF8B92001F097F8BB20F5
:104FA00001F094F8B22001F091F842E0B32001F052
:104FB0008DF8AB2001F08AF8B12001F087F8B0201D
:104FC000FEF7E4FDB920FEF7E1FDBB20FEF7DEFDB4
:104FD000B220FEF7DBFD2CE0B32001F077F8AB2028
:104FE00001F074F8B12001F071F8B02001F06EF812
:104FF000B92001F06BF8BB2001F068F8B22001F095
:1050000065F816E0B32001F061F8AB2001F05EF81E
:10501000B12001F05BF8B02001F058F8B920FEF79C
:10502000B5FDBB2001F052F8B22001F04FF800E0CE
:1050300000BF00BF5EE4230002F033FC0A061C320E
:10504000485E748AA0B6CCE2A32001F03FF89A2013
:1050500001F03CF8992001F039F8A02001F036F871
:10506000A92001F033F8A22001F030F8A120FEF7CA
:105070008DFDC6E0A320FEF789FD9A2001F026F8F9
:10508000992001F023F8A020FEF780FDA920FEF76B
:105090007DFDA220FEF77AFDA120FEF777FDB0E0AE
:1050A000A32001F013F89A2001F010F89920FEF7E0
:1050B0006DFDA02001F00AF8A92001F007F8A22058
:1050C000FEF764FDA12001F001F89AE0A32000F0B2
:1050D000FDFF9A2000F0FAFF992000F0F7FFA020D2
:1050E00000F0F4FFA920FEF751FDA220FEF74EFDCF
:1050F000A12000F0EBFF84E0A320FEF747FD9A20FB
:1051000000F0E4FF992000F0E1FFA020FEF73EFD53
:10511000A920FEF73BFDA22000F0D8FFA12000F05F
:10512000D5FF6EE0A32000F0D1FF9A20FEF72EFD00
:10513000992000F0CBFFA02000F0C8FFA920FEF7C7
:1051400025FDA22000F0C2FFA12000F0BFFF58E023
:10515000A32000F0BBFF9A20FEF718FD992000F075
:10516000B5FFA02000F0B2FFA92000F0AFFFA22001
:1051700000F0ACFFA12000F0A9FF42E0A32000F066
:10518000A5FF9A2000F0A2FF992000F09FFFA02029
:10519000FEF7FCFCA920FEF7F9FCA220FEF7F6FCC6
:1051A000A120FEF7F3FC2CE0A32000F08FFF9A2053
:1051B00000F08CFF992000F089FFA02000F086FF0E
:1051C000A92000F083FFA22000F080FFA12000F0C2
:1051D0007DFF16E0A32000F079FF9A2000F076FF13
:1051E000992000F073FFA02000F070FFA920FEF7C7
:1051F000CDFCA22000F06AFFA12000F067FF00E0D4
:1052000000BF00BF5EE4230002F04BFB0A061C3225
:10521000485E748AA0B6CCE2932000F057FF8A2043
:1052200000F054FF882000F051FF902000F04EFF66
:10523000912000F04BFF922000F048FF8920FEF7FC
:10524000A5FCC6E09320FEF7A1FC8A2000F03EFFFB
:10525000882000F03BFF9020FEF798FC9120FEF79D
:1052600095FC9220FEF792FC8920FEF78FFCB0E0BF
:10527000932000F02BFF8A2000F028FF8820FEF703
:1052800085FC902000F022FF912000F01FFF92206B
:10529000FEF77CFC892000F019FF9AE0932000F0D3
:1052A00015FF8A2000F012FF882000F00FFF9020E9
:1052B00000F00CFF9120FEF769FC9220FEF766FCDF
:1052C000892000F003FF84E09320FEF75FFC8A2032
:1052D00000F0FCFE882000F0F9FE9020FEF756FC5E
:1052E0009120FEF753FC922000F0F0FE892000F0A0
:1052F000EDFE6EE0932000F0E9FE8A20FEF746FC0A
:10530000882000F0E3FE902000F0E0FE9120FEF700
:105310003DFC922000F0DAFE892000F0D7FE58E034
:10532000932000F0D3FE8A20FEF730FC882000F0A6
:10533000CDFE902000F0CAFE912000F0C7FE922022
:1053400000F0C4FE892000F0C1FE42E0932000F08E
:10535000BDFE8A2000F0BAFE882000F0B7FE902043
:10536000FEF714FC9120FEF711FC9220FEF70EFCD4
:105370008920FEF70BFC2CE0932000F0A7FE8A208A
:1053800000F0A4FE882000F0A1FE902000F09EFE18
:10539000912000F09BFE922000F098FE892000F002
:1053A00095FE16E0932000F091FE8A2000F08EFE1C
:1053B000882000F08BFE902000F088FE9120FEF700
:1053C000E5FB922000F082FE892000F07FFE00E0E5
:1053D00000BF00BF5EE4230002F063FA0A061F3834
:1053E000516A839CB5CEE7FDFC2000F06FFEFD20E6
:1053F00000F06CFEFE2000F069FEFF2000F066FE6B
:10540000FF20083000F062FEFF20063000F05EFE54
:10541000FF200730FEF7BAFBE3E0FC20FEF7B6FB07
:10542000FD2000F053FEFE2000F050FEFF20FEF7AE
:10543000ADFBFF200830FEF7A9FBFF200630FEF78A
:10544000A5FBFF200730FEF7A1FBCAE0FC2000F01F
:105450003DFEFD2000F03AFEFE20FEF797FBFF2008
:1054600000F034FEFF20083000F030FEFF20063050
:10547000FEF78CFBFF20073000F028FEB1E0FC2097
:1054800000F024FEFD2000F021FEFE2000F01EFEB4
:10549000FF2000F01BFEFF200830FEF777FBFF2007
:1054A0000630FEF773FBFF20073000F00FFE98E098
:1054B000FC20FEF76BFBFD2000F008FEFE2000F054
:1054C00005FEFF20FEF762FBFF200830FEF75EFBC3
:1054D000FF20063000F0FAFDFF20073000F0F6FD57
:1054E0007FE0FC2000F0F2FDFD20FEF74FFBFE20E8
:1054F00000F0ECFDFF2000F0E9FDFF200830FEF792
:1055000045FBFF20063000F0E1FDFF20073000F0F2
:10551000DDFD66E0FC2000F0D9FDFD20FEF736FB46
:10552000FE2000F0D3FDFF2000F0D0FDFF2008306A
:1055300000F0CCFDFF20063000F0C8FDFF20073052
:1055400000F0C4FD4DE0FC2000F0C0FDFD2000F0A7
:10555000BDFDFE2000F0BAFDFF20FEF717FBFF2087
:105560000830FEF713FBFF200630FEF70FFBFF208D
:105570000730FEF70BFB34E0FC2000F0A7FDFD2018
:1055800000F0A4FDFE2000F0A1FDFF2000F09EFD34
:10559000FF20083000F09AFDFF20063000F096FD55
:1055A000FF20073000F092FD1BE0FC2000F08EFD94
:1055B000FD2000F08BFDFE2000F088FDFF2000F0B4
:1055C00085FDFF200830FEF7E1FAFF20063000F0ED
:1055D0007DFDFF2000E003E0073000F077FD00E0F4
:1055E00000BF00BF3EE4230002F05BF90A061C3254
:1055F000485E748AA0B6CCE2EC2000F067FDE4209F
:1056000000F064FDEE2000F061FDEF2000F05EFD93
:10561000F62000F05BFDF42000F058FDED20FEF7D1
:10562000B5FAC6E0EC20FEF7B1FAE42000F04EFD3A
:10563000EE2000F04BFDEF20FEF7A8FAF620FEF773
:10564000A5FAF420FEF7A2FAED20FEF79FFAB0E0EB
:10565000EC2000F03BFDE42000F038FDEE20FEF7EA
:1056600095FAEF2000F032FDF62000F02FFDF42037
:10567000FEF78CFAED2000F029FD9AE0EC2000F016
:1056800025FDE42000F022FDEE2000F01FFDEF20BC
:1056900000F01CFDF620FEF779FAF420FEF776FA0A
:1056A000ED2000F013FD84E0EC20FEF76FFAE4201B
:1056B00000F00CFDEE2000F009FDEF20FEF766FA89
:1056C000F620FEF763FAF42000F000FDED2000F074
:1056D000FDFC6EE0EC2000F0F9FCE420FEF756FA49
:1056E000EE2000F0F3FCEF2000F0F0FCF620FEF7D7
:1056F0004DFAF42000F0EAFCED2000F0E7FC58E061
:10570000EC2000F0E3FCE420FEF740FAEE2000F08D
:10571000DDFCEF2000F0DAFCF62000F0D7FCF420EE
:1057200000F0D4FCED2000F0D1FC42E0EC2000F0D1
:10573000CDFCE42000F0CAFCEE2000F0C7FCEF2016
:10574000FEF724FAF620FEF721FAF420FEF71EFAFF
:10575000ED20FEF71BFA2CE0EC2000F0B7FCE42073
:1057600000F0B4FCEE2000F0B1FCEF2000F0AEFC45
:10577000F62000F0ABFCF42000F0A8FCED2000F0D7
:10578000A5FC16E0EC2000F0A1FCE42000F09EFC5B
:10579000EE2000F09BFCEF2000F098FCF620FEF7D6
:1057A000F5F9F42000F092FCED2000F08FFC00E011
:1057B00000BF00BF3EE4230002F073F80A061C326B
:1057C000485E748AA0B6CCE2DC2000F07FFCD520D5
:1057D00000F07CFCD62000F079FCDF2000F076FCA5
:1057E000E62000F073FCDD2000F070FCDE20FEF708
:1057F000CDF9C6E0DC20FEF7C9F9D52000F066FC43
:10580000D62000F063FCDF20FEF7C0F9E620FEF7AB
:10581000BDF9DD20FEF7BAF9DE20FEF7B7F9B0E0FA
:10582000DC2000F053FCD52000F050FCD620FEF721
:10583000ADF9DF2000F04AFCE62000F047FCDD2057
:10584000FEF7A4F9DE2000F041FC9AE0DC2000F035
:105850003DFCD52000F03AFCD62000F037FCDF20DC
:1058600000F034FCE620FEF791F9DD20FEF78EF91A
:10587000DE2000F02BFC84E0DC20FEF787F9D52049
:1058800000F024FCD62000F021FCDF20FEF77EF99A
:10589000E620FEF77BF9DD2000F018FCDE2000F0AA
:1058A00015FC6EE0DC2000F011FCD520FEF76EF94F
:1058B000D62000F00BFCDF2000F008FCE620FEF70D
:1058C00065F9DD2000F002FCDE2000F0FFFB58E06F
:1058D000DC2000F0FBFBD520FEF758F9D62000F0C5
:1058E000F5FBDF2000F0F2FBE62000F0EFFBDD200F
:1058F00000F0ECFBDE2000F0E9FB42E0DC2000F0F1
:10590000E5FBD52000F0E2FBD62000F0DFFBDF2036
:10591000FEF73CF9E620FEF739F9DD20FEF736F90F
:10592000DE20FEF733F92CE0DC2000F0CFFBD520A1
:1059300000F0CCFBD62000F0C9FBDF2000F0C6FB56
:10594000E62000F0C3FBDD2000F0C0FBDE2000F00D
:10595000BDFB16E0DC2000F0B9FBD52000F0B6FB63
:10596000D62000F0B3FBDF2000F0B0FBE620FEF70E
:105970000DF9DD2000F0AAFBDE2000F0A7FB00E01F
:1059800000BF00BF9FE3230001F08BFF0A061C321B
:10599000485E748AA0B6CCE2CC2000F097FBC5200C
:1059A00000F094FBC72000F091FBCF2000F08EFBAD
:1059B000CE2000F08BFBCD2000F088FBC620FEF748
:1059C000E5F8C6E0CC20FEF7E1F8C52000F07EFB4C
:1059D000C72000F07BFBCF20FEF7D8F8CE20FEF7E3
:1059E000D5F8CD20FEF7D2F8C620FEF7CFF8B0E00C
:1059F000CC2000F06BFBC52000F068FBC720FEF751
:105A0000C5F8CF2000F062FBCE2000F05FFBCD2078
:105A1000FEF7BCF8C62000F059FB9AE0CC2000F05D
:105A200055FBC52000F052FBC72000F04FFBCF20F4
:105A300000F04CFBCE20FEF7A9F8CD20FEF7A6F82B
:105A4000C62000F043FB84E0CC20FEF79FF8C52081
:105A500000F03CFBC72000F039FBCF20FEF796F8A2
:105A6000CE20FEF793F8CD2000F030FBC62000F0EA
:105A70002DFB6EE0CC2000F029FBC520FEF786F858
:105A8000C72000F023FBCF2000F020FBCE20FEF744
:105A90007DF8CD2000F01AFBC62000F017FB58E07F
:105AA000CC2000F013FBC520FEF770F8C72000F0F3
:105AB0000DFBCF2000F00AFBCE2000F007FBCD202D
:105AC00000F004FBC62000F001FB42E0CC2000F017
:105AD000FDFAC52000F0FAFAC72000F0F7FACF204F
:105AE000FEF754F8CE20FEF751F8CD20FEF74EF821
:105AF000C620FEF74BF82CE0CC2000F0E7FAC520DA
:105B000000F0E4FAC72000F0E1FACF2000F0DEFA5E
:105B1000CE2000F0DBFACD2000F0D8FAC62000F04D
:105B2000D5FA16E0CC2000F0D1FAC52000F0CEFA6C
:105B3000C72000F0CBFACF2000F0C8FACE20FEF745
:105B400025F8CD2000F0C2FAC62000F0BFFA00E030
:105B500000BF00BFB7E2230001F0A3FE0A061C321B
:105B6000485E748AA0B6CCE2B42000F0AFFAB5204B
:105B700000F0ACFAB62000F0A9FAB72000F0A6FABF
:105B8000BE2000F0A3FABC2000F0A0FABD20FDF773
:105B9000FDFFC6E0B420FDF7F9FFB52000F096FA4E
:105BA000B62000F093FAB720FDF7F0FFBE20FDF716
:105BB000EDFFBC20FDF7EAFFBD20FDF7E7FFB0E0F9
:105BC000B42000F083FAB52000F080FAB620FDF78B
:105BD000DDFFB72000F07AFABE2000F077FABC2093
:105BE000FDF7D4FFBD2000F071FA9AE0B42000F078
:105BF0006DFAB52000F06AFAB62000F067FAB72017
:105C000000F064FABE20FDF7C1FFBC20FDF7BEFF27
:105C1000BD2000F05BFA84E0B420FDF7B7FFB520AB
:105C200000F054FAB62000F051FAB720FDF7AEFFAD
:105C3000BE20FDF7ABFFBC2000F048FABD2000F00D
:105C400045FA6EE0B42000F041FAB520FDF79EFF62
:105C5000B62000F03BFAB72000F038FABE20FDF77E
:105C600095FFBC2000F032FABD2000F02FFA58E07A
:105C7000B42000F02BFAB520FDF788FFB62000F025
:105C800025FAB72000F022FABE2000F01FFABC204F
:105C900000F01CFABD2000F019FA42E0B42000F038
:105CA00015FAB52000F012FAB62000F00FFAB7206E
:105CB000FDF76CFFBE20FDF769FFBC20FDF766FF16
:105CC000BD20FDF763FF2CE0B42000F0FFF9B52004
:105CD00000F0FCF9B62000F0F9F9B72000F0F6F971
:105CE000BE2000F0F3F9BC2000F0F0F9BD2000F078
:105CF000EDF916E0B42000F0E9F9B52000F0E6F97E
:105D0000B62000F0E3F9B72000F0E0F9BE20FDF77F
:105D10003DFFBC2000F0DAF9BD2000F0D7F900E02B
:105D200000BF00BFCFE1230001F0BBFD0A061C321B
:105D3000485E748AA0B6CCE2A42000F0C7F99C208B
:105D400000F0C4F9A62000F0C1F9A72000F0BEF9C8
:105D5000AE2000F0BBF9AC2000F0B8F9A520FDF7AB
:105D600015FFC6E0A420FDF711FF9C2000F0AEF95E
:105D7000A62000F0ABF9A720FDF708FFAE20FDF745
:105D800005FFAC20FDF702FFA520FDF7FFFEB0E008
:105D9000A42000F09BF99C2000F098F9A620FDF7C4
:105DA000F5FEA72000F092F9AE2000F08FF9AC20AC
:105DB000FDF7ECFEA52000F089F99AE0A42000F0A0
:105DC00085F99C2000F082F9A62000F07FF9A72039
:105DD00000F07CF9AE20FDF7D9FEAC20FDF7D6FE31
:105DE000A52000F073F984E0A420FDF7CFFE9C20ED
:105DF00000F06CF9A62000F069F9A720FDF7C6FEB7
:105E0000AE20FDF7C3FEAC2000F060F9A52000F045
:105E10005DF96EE0A42000F059F99C20FDF7B6FE74
:105E2000A62000F053F9A72000F050F9AE20FDF7AE
:105E3000ADFEAC2000F04AF9A52000F047F958E08B
:105E4000A42000F043F99C20FDF7A0FEA62000F05E
:105E50003DF9A72000F03AF9AE2000F037F9AC2068
:105E600000F034F9A52000F031F942E0A42000F060
:105E70002DF99C2000F02AF9A62000F027F9A72090
:105E8000FDF784FEAE20FDF781FEAC20FDF77EFE1F
:105E9000A520FDF77BFE2CE0A42000F017F99C2044
:105EA00000F014F9A62000F011F9A72000F00EF977
:105EB000AE2000F00BF9AC2000F008F9A52000F0AE
:105EC00005F916E0A42000F001F99C2000F0FEF88E
:105ED000A62000F0FBF8A72000F0F8F8AE20FDF7B0
:105EE00055FEAC2000F0F2F8A52000F0EFF800E03D
:105EF00000BF00BFE7E0230001F0D3FC0A061C321C
:105F0000485E748AA0B6CCE2942000F0DFF88D20C1
:105F100000F0DCF88F2000F0D9F8972000F0D6F8D8
:105F20009E2000F0D3F8952000F0D0F89620FDF7E1
:105F30002DFEC6E09420FDF729FE8D2000F0C6F866
:105F40008F2000F0C3F89720FDF720FE9E20FDF77C
:105F50001DFE9520FDF71AFE9620FDF717FEB0E016
:105F6000942000F0B3F88D2000F0B0F88F20FDF7FA
:105F70000DFE972000F0AAF89E2000F0A7F89520CB
:105F8000FDF704FE962000F0A1F89AE0942000F0BE
:105F90009DF88D2000F09AF88F2000F097F8972058
:105FA00000F094F89E20FDF7F1FD9520FDF7EEFD41
:105FB000962000F08BF884E09420FDF7E7FD8D201B
:105FC00000F084F88F2000F081F89720FDF7DEFDC7
:105FD0009E20FDF7DBFD952000F078F8962000F07C
:105FE00075F86EE0942000F071F88D20FDF7CEFD7D
:105FF0008F2000F06BF8972000F068F89E20FDF7E6
:10600000C5FD952000F062F8962000F05FF858E09A
:10601000942000F05BF88D20FDF7B8FD8F2000F094
:1060200055F8972000F052F89E2000F04FF8952088
:1060300000F04CF8962000F049F842E0942000F07F
:1060400045F88D2000F042F88F2000F03FF89720AF
:10605000FDF79CFD9E20FDF799FD9520FDF796FD2F
:106060009620FDF793FD2CE0942000F02FF88D2072
:1060700000F02CF88F2000F029F8972000F026F887
:106080009E2000F023F8952000F020F8962000F0E4
:106090001DF816E0942000F019F88D2000F016F895
:1060A0008F2000F013F8972000F010F89E20FDF7E5
:1060B0006DFD952000F00AF8962000F007F800E04A
:1060C00000BF00BF00BF00BF70BD000030B501467B
:1060D000C3175B0F5B18DB10094CE35C0246C41767
:1060E000640FA418E410E400051B0124AC40234312
:1060F000C417640F6418E410014D2B5530BD000027
:106100009620002010B5044630222146002000F0E1
:10611000F2F810BD10B500F067FE08210C48FCF73E
:106120005CFA012002F0FAFB04210948FCF757FA57
:10613000042002F0F3FB04210548FCF74EFA04208A
:1061400002F0ECFB08210248FCF749FA10BD000000
:10615000C00C004010B500F047FE08210A48FCF7CB
:106160003EFA012002F0DAFB04210748FCF737FA77
:10617000042002F0D3FB04210348FCF72EFA04208C
:1061800002F0CCFB10BD0000C00C004070B5002533
:1061900008211348FCF723FA00F016FE80241BE0C8
:1061A00004210F48FCF71BFA012002F0B7FB08217D
:1061B0000B48FCF708FA012803D12846204305467E
:1061C00002E02846A043054604210548FCF705FAED
:1061D000042002F0A3FB6410002CE1D1284670BD1E
:1061E000C00C004070B5044600F0FEFD00251EE026
:1061F00080202040002804D008211548FCF7EFF942
:1062000003E008211248FCF7E8F96006040E0A20B2
:1062100002F084FB04210E48FCF7E1F90A2002F0A9
:106220007DFB04210A48FCF7D8F9681CC5B2082D8B
:10623000DEDB0A2002F072FB04210548FCF7CFF9EF
:106240000A2002F06BFB04210148FCF7C6F970BD7F
:10625000C00C004010B500F0C7FD08210A48FCF74B
:10626000BEF904210848FCF7BAF9052002F056FBF4
:1062700008210548FCF7B1F9042002F04FFB042186
:106280000148FCF7AAF910BDC00C004010B500F0A1
:10629000ABFD08210A48FCF7A0F9042002F03EFB00
:1062A00004210748FCF79BF9042002F037FB082182
:1062B0000348FCF794F9052002F030FB10BD000004
:1062C000C00C0040F8B507460D4616460024FFF7FF
:1062D000C1FF7C20FFF786FF3846FFF783FF00BF32
:1062E00004E0285DFFF77EFF601CC4B2B442F8DB17
:1062F000FFF7CCFFF8BDF8B507460D46164600245B
:10630000FFF7A8FF7C20FFF76DFF8020FFF76AFFF3
:106310003846FFF767FF00BF04E0285DFFF762FF24
:10632000601CC4B2B442F8DBFFF7B0FFF8BD08B59B
:10633000022002F0CBFA032168460170012269466F
:106340008220FFF7BFFF032168460170022002F0A0
:10635000BDFA012269468420FFF7B4FF08BD0000A2
:1063600004488069C007C00F002801D00120704791
:106370000020FCE70034014010B500F00BF80128C4
:1063800007D1FFF7EDFF012803D100F00FF802F06D
:10639000C3F810BD0448406940210840002801D0DE
:1063A000012070470020FCE70034014040200149F3
:1063B000486170470034014000200C4909780029E9
:1063C00003D00A490978092901D101210843084964
:1063D00089784907490F042907D005498978490771
:1063E000490F032901D002210843704714000020FF
:1063F0001C010020F0B589B00021C848C1720173AA
:10640000002600250CE0C648405D412807D1C4485D
:10641000691C405C412802D1C148461964256D1CA5
:10642000642DF0DB002E38D00027002507E0705DDA
:10643000BC4948550846405DC019C7B26D1C192DAE
:10644000F5DB707EB84228D1B07E162825D1B07811
:10645000012816D1F078012802DDF078B249C87120
:10646000002504E0301D415DB04841556D1C142DE0
:10647000F8DB307E002805D0317EAB4820308171BA
:1064800000E000BF0120A8494870032088707821EF
:10649000A5482330017100214171A5A1A048F9F759
:1064A000ABFE0646002E7DD0A2A13046F9F7A4FE31
:1064B0000446002CF7D00025641C04E06D1C641C0D
:1064C0000A2D00DD02E060786828F7D100BF78214E
:1064D00095482330017100214171E07A0690207BBC
:1064E000617B0902401880B20790607DA17D09029E
:1064F000401880B20890E07E05900027002504E057
:10650000601C405DC019C7B26D1C07980D308542F4
:10651000F6DB07982018807BB84243D16078682862
:10652000FBD1A07A6828F8D1FCF78EFA82488079EE
:106530007E491C3948738048C07888737E4800794A
:10654000C8737D48007808747B48407848747A485E
:1065500080788874069805284ED178490898884232
:106560004AD1802105980840002803D1207F0028C7
:1065700014D013E0002505E020461C30405D694939
:1065800048556D1C102DF7DB664A6D491046FAF729
:10659000E5FB64480078002800D000BF63491C393F
:1065A000C87D00E0B8E0897D000208435F4A1C3ADC
:1065B000517E127E09021143884203DA00215A48B3
:1065C0002030417259491C39C87D897D0002084339
:1065D000401C80B255491C398875000AC875594855
:1065E0000078042805DB57480078001F55490870DB
:1065F00002E0002053490870069801288DD15249C5
:106600000898884289D14C484078A17C884210DCA7
:10661000A17C49484078C01C81421ADD4648407838
:106620006030A17C401A092813DD01204749087019
:106630000FE041484178A07CC01C814209DDA07C6C
:1066400060303D494978401A092802DD01203F4960
:1066500008703E480078012825D1A07B3C4908708D
:10666000E07B4870207C8870607CC870A07C0871DA
:10667000E07C4871084640790979354AD278009221
:106680000191029032488278407804903048007836
:1066900001214903401801230390049900F018FCDC
:1066A00000202A4908702BA0FCF79EF8FF20F53047
:1066B00002F00CF9FF20F53002F008F9FF20F53068
:1066C00002F004F9FF20F53002F000F9FF2101315A
:1066D0002248F9F786FDFF2101311148F9F781FDC4
:1066E00000210E48C17201730F4820304172002012
:1066F0001449087001210D481C3881750021C175AD
:1067000000201749087017490870174908700021C0
:10671000154820308174C17409B0F0BD771D002088
:10672000771C00203F1E0020881D0020CF1D002068
:106730002B5200002C0000001A060020608400008C
:10674000481700200F06002050A400003506002046
:10675000220600204154434C4F534500771B002034
:106760000206002004060020711A002070B50446BD
:106770000025FCF7DDFB1048007C002819D0002123
:106780000D480174FF210131401AF9F72AFD0A482A
:10679000C27A0A49FF380138F9F70AFD122C02D1F2
:1067A000FFF728FE04E000210348C172017300BF17
:1067B00000BF284670BD0000771D0020771B002019
:1067C000002805DBC206D20E01219140014A11606A
:1067D0007047000080E100E0002805DBC206D20E11
:1067E00001219140014A11607047000000E100E082
:1067F00010B5002819DB1A4A03231B02D21883089C
:106800009B00D2588307DC0EFF23A3409A438B07DB
:106810001B0E8407E40EA3401A43114B03242402E9
:106820001B198408A4001A5118E00E4A03071B0F15
:10683000083B9B089B00D2588307DC0EFF23A34034
:106840009A438B071B0E8407E40EA3401A43054BA3
:106850000407240F083CA408A4001A5110BD00002E
:1068600000E100E01CED00E07FB506460D46144651
:106870006A4629463046FBF7A9FD0098A84217D181
:106880006846C079002813D1002C03D168464079AE
:1068900000280DD1012C03D168464079012807D189
:1068A00068468079002803D168460079012813D012
:1068B000029500206946C873002C01D1487302E09C
:1068C00001206946487300216846817301210173E4
:1068D00002A93046FBF73EFE7FBD00000146064A96
:1068E0001068931502469A4310461A460A40104310
:1068F000014A106070470000002000400146054A30
:106900001068800880008A07920F1043014A1060C7
:1069100070470000002000400146064A10685315E9
:1069200002469A4310461A460A401043014A106034
:10693000704700000020004010B504466068FFF773
:10694000EBFF207AFFF7CAFF012149026068884205
:1069500002D1206900F00AF80349E0680861206864
:10696000FFF7CCFF10BD000000ED00E00146054A36
:106970005068800880008A07920F1043014A5060D7
:10698000704700000020004010B502F067F902F0E7
:10699000A5F902F013FA02F0BBFA02F023FB00F0B3
:1069A00005F802F085F9FCF707FB10BD10B50821CA
:1069B0003048FBF708FE00281CD104212D48FBF7C6
:1069C0000CFE002414E0FF2101312A48C038FBF7F7
:1069D00004FEC82001F07AFFFF2101312548C038AC
:1069E000FBF7FDFDC82001F071FFFCF7E5FA641C20
:1069F000032CE8DB02211F48C038FBF7E4FD012827
:106A000037D1002414E0FF2101311A48C038FBF7C8
:106A1000E4FDC82001F05AFFFF2101311548C038BC
:106A2000FBF7DDFDC82001F051FFFCF7C5FA641C3F
:106A3000052CE8DB80210F48FBF7C5FD012818D1A4
:106A4000002414E0FF2101310A48C038FBF7C5FDDE
:106A5000C82001F03BFFFF2101310648C038FBF799
:106A6000BEFDC82001F032FFFCF7A6FA641C062C1C
:106A7000E8DB10BD800D0040F8B507460D46164610
:106A8000FFF7E8FB6420FFF7ADFB3846FFF7AAFBF2
:106A9000FFF7E0FB6520FFF7A5FB002406E0FFF70A
:106AA00075FB2855FFF736FB601CC4B2701EA04270
:106AB000F5DCFFF76BFB2855FFF74CFBFFF7E6FB18
:106AC000F8BDF8B507460D461646FFF7C3FB642030
:106AD000FFF788FB3846FFF785FB002404E0285DBC
:106AE000FFF780FB601CC4B2B442F8DBFFF7CEFBBB
:106AF000F8BD00000146064A5068062302469A4344
:106B0000104606220A401043014A506070470000B8
:106B100000280040012806D1064949680122114396
:106B2000044A516005E00349496849084900014A9F
:106B300051607047002800400146064A106806234D
:106B400002469A43104606220A401043014A10604A
:106B50007047000000280040012806D10649096856
:106B600001221143044A116005E0034909684908FC
:106B70004900014A1160704700280040C104C90C57
:106B8000014A11637047000000100140024880690B
:106B90008006800E704700000010014002484069E6
:106BA0008006800E70470000001001400248006916
:106BB0004006400E70470000001001400248006A85
:106BC000C006C00E70470000001001400248C068B7
:106BD0004006400E70470000001001400248C069A6
:106BE0004007400F70470000001001400148406A14
:106BF000C0B270470010014010B501210648FAF7F5
:106C0000B5FD002204210548FFF72EFE00220821D1
:106C10000248FFF729FE10BD07000001C00C00402C
:106C200010B50B48407A012805D1FFF7C5FB0328B2
:106C300001D100F0E9F800F011F8012807D100F0C7
:106C400019F80120034908700348FBF7CBFE10BD7B
:106C5000E40300203C040020050000200448806874
:106C600008210840002801D0012070470020FCE7DF
:106C70000010014008200149886070470010014061
:106C800000B50146FFF7A2FF4871FFF78FFF0871BB
:106C9000FFF784FFC870FFF779FF8870FFF78EFF5A
:106CA0004870FFF7A3FF0870FFF798FF887100BDD9
:106CB00010B500F065F8012828D1022024490861A8
:106CC00000F06AF800BF234800798007C00F002851
:106CD00012D12049097C02229143891C1D4A11745A
:106CE0008907C90F4900022211400846194909794C
:106CF00091430143174A117100BF012016490870E2
:106D00000020C87315A000F091FD1FE000F04AF8C4
:106D100001281BD10E49086100F050F800BF0D4852
:106D200000798007C00F00280CD00A4800790221A2
:106D300088430849087111200B49088011210B482C
:106D4000FAF77EF800BF0AA000F070FD10BD000049
:106D5000002801401C010020FA000020EFAEB5E73A
:106D6000C7B7D1B90D0A0000F800002028040020A0
:106D7000EFAEB5E7C7B7D1B9BBD6B8B40D0A0000BE
:106D80000448C06802210840002801D00120704753
:106D90000020FCE70028014002200149C86070473C
:106DA000002801400448C068C007C00F002801D077
:106DB000012070470020FCE7002801400120014924
:106DC000C86070470028014010B501210448FAF757
:106DD000CDFC002208210348FCF781F910BD00001A
:106DE00007000001C00C004010B501210448FAF76B
:106DF000BDFC002208210348FFF736FD10BD00004E
:106E000007000001C00C00401FB500240120FAF764
:106E1000B5FD07200002FAF7C3FD032001F056FD7F
:106E20000120FAF7DDFB05E019200002844200D3BF
:106E300004E0641CFAF7E8FB0028F5D000BF01204D
:106E40000090002001900290012069460873684676
:106E5000FAF784FD014801F015FD1FBD001BB700C6
:106E60000148006870470000B00300200148024953
:106E70000860704700127A003806002010B572B61C
:106E8000FCF7A2F8104801F0FDFC0A2001F01EFDFD
:106E9000FCF71AF90120FFF75FFE0620FFF72AFE34
:106EA0000020FFF737FEFAF72EFE01210748FAF718
:106EB0005DFC0020FFF762FE00210448FAF756FC53
:106EC000FCF77AF862B610BD00127A0002000001E9
:106ED000FFB583B006460C4615460C9F0120474976
:106EE0000870FFF789FEF6B2F0210E9808400011F5
:106EF0000A2148430E990907090F40183C2803DA74
:106F000069460E98087102E0002069460871F02178
:106F10000D98084000110A2148430D990907090FEF
:106F200040183C2803DA69460D98487102E00020B9
:106F300069464871F020384000110A21484339075A
:106F4000090F4018182802DA6846877102E000200D
:106F50006946887169460698C871F020284000117A
:106F60000A2148432907090F401820280CDAF0208D
:106F7000284000110A2148432907090F401800281A
:106F800002DD6846057202E0012069460872F020C1
:106F9000204000110A2148432107090F40180D28FD
:106FA0000CDAF020204000110A2148432107090F84
:106FB0004018002802DD6846447202E0012069465C
:106FC0004872F020304000110A2148433107090F70
:106FD0004018642802DA69468E7202E0152069467C
:106FE0008872072201A90020FFF76BFD0A2001F03B
:106FF0006DFC00200149087007B0F0BD3606002086
:1070000070B504460D4601218806FAF7AFFB032050
:10701000FAF79EFB0120FAF789FB0120FAF75EF9E7
:107020000020FAF77FF9601EFAF7C0F9681EFAF738
:107030004FF91B20FFF7C4FB01211B20FFF7D8FBF2
:107040001B20FFF7C9FB0120FAF77CF90120FAF7B2
:1070500057F9FAF7A5F970BD10B5044800F021FB07
:10706000012802D1014800F027FB10BD0068014053
:1070700010B5044800F015FB012802D1014800F0CA
:107080001BFB10BD00780140F3B585B00F46059895
:10709000F9F746FB05463846F9F742FB064629460E
:1070A000F9F76EF904907F21C9050498F9F708FCF7
:1070B00013D20498F9F7C0FB05460022094BF9F7F3
:1070C00041FA0022084B01910090F9F797F90391DA
:1070D0000290F9F773FB044600E00024204607B055
:1070E000F0BD00000000F03F0000E03F30B5054675
:1070F0000C462846616800F01FFA2846A16800F097
:107100002AFA2846E16800F01AFA2846616900F078
:1071100053FA617C284600F08EFA217C284600F064
:1071200097FA2178284600F079FA6178284600F02D
:107130009CFAA178284600F0A4FAA17E284600F027
:1071400022FAE17E284600F05DFAA17C284600F094
:107150000EFA217E284600F03CFA617E284600F0B7
:1071600044FA30BD00B597B001216648FAF7FEFA3F
:107170000022FF2101316448F9F788FF0022012134
:1071800049026148F9F782FF0022012189025E4825
:10719000FFF76AFB012189025B48FBF720FAE12037
:1071A00040021490012110A80175002141758175DC
:1071B0000DA8FAF785F90DAA14A9544800F0B4F8FF
:1071C0000E20FFF7FDFA0121504800F0D0F901210F
:1071D0004E4800F0FEF94D4800F05FFA01214C489E
:1071E000FAF7C4FA0120FAF7EDFD052168460171AE
:1071F000012040030390801004900320400205907A
:1072000000200690434802904348099000200790D0
:10721000002108A8417081700121C1701520FFF77D
:10722000CFFA0520FAF7E0FD01A8FAF7E5FD012104
:107230003748FAF79BFA0120FAF7C4FD01213148DB
:10724000FAF794FA002208213448F9F71FFF0022C8
:1072500010213248F9F71AFF00201690E120400271
:107260001490012110A801750021417581750DA8A8
:10727000FAF726F90DAA14A9294800F055F80A20B2
:10728000FFF79EFAFF21264800F070FA244800F02C
:1072900013FA0121224800F0DBF90A20FFF79CFADB
:1072A00001211F4800F07BF901211D4800F05FF922
:1072B00001211B4800F08DF9194800F0EEF9032177
:1072C0006846017101204003039080100490080279
:1072D0000590002006900F48029012480990002067
:1072E0000790002108A8417081700121C17015200C
:1072F000FFF766FA0320FAF777FD01A8FAF77CFD9D
:1073000017B000BD07000001000C004000780140EC
:1073100004000002FF03000048060020000D0040AA
:10732000006801404412002070B588B006460C4643
:1073300015467A48864228D1A068FAF7C5F9012097
:10734000FAF7AEF901217648FAF710FAA06800289A
:1073500004D0012808D0022815D10EE0A9682068C1
:10736000FFF792FE02900FE00120FAF775FAE96844
:107370002068FFF789FE029006E029682068FFF781
:1073800083FE029000E000BF63E06648864229D198
:10739000A068FAF7BBF90120FAF7A4F901216048C7
:1073A000401CFAF7E3F9A068002804D0042808D0AC
:1073B000082815D10EE0A9682068FFF765FE029045
:1073C0000FE00120FAF748FAE9682068FFF75CFE51
:1073D000029006E029682068FFF756FE029000E060
:1073E00000BF36E0504886420AD101214C48801C3B
:1073F000FAF7BCF9A9682068FFF746FE029028E07A
:107400004A4886420AD101214548C01CFAF7AEF924
:10741000A9682068FFF738FE02901AE044488642C7
:107420000AD101213E48001DFAF7A0F9A968206899
:10743000FFF72AFE02900CE03E48864209D1012166
:107440003748401DFAF792F9A9682068FFF71CFE3B
:1074500002902079012810D1402003906079012802
:1074600002D1102004903FE06079022802D1202050
:10747000049039E00020049036E02079022810D1F1
:10748000802003906079012802D1102004902BE025
:107490006079022802D12020049025E00020049089
:1074A00022E0207900280FD103906079012802D1D1
:1074B0001020049018E06079022802D12020049066
:1074C00012E0002004900FE0C020039060790128B2
:1074D00002D11020049007E06079022802D1202018
:1074E000049001E000200490A079002801D10690CA
:1074F00002E0FF20013006900021684601714171D1
:107500008171417501758177C17781750177417707
:1075100001A93046FFF7EAFD08B070BD0020014028
:107520000800000300680140006C01400070014049
:1075300000740140007801408AB28261704710B542
:107540000A46016830240B46A343194630231340F2
:107550001943016010BD10B50A460168C0240B46EE
:10756000A3431946C02313401943016010BD0129EC
:1075700004D1026802231A43026003E00268022376
:107580009A4302607047012904D1026808231A4314
:10759000026003E0026808239A43026070470129F1
:1075A00004D102680B041A43026004E0026801235C
:1075B0001B049A430260704710B50A460168FF2415
:1075C00001340B46A3431946234613401943016077
:1075D00010BD012904D1026801231A43026003E0AF
:1075E00002685208520002607047012904D1026803
:1075F0004B041A43026004E0026801235B049A43CF
:1076000002607047012904D1026804231A43026012
:1076100003E0026804239A4302607047012904D101
:1076200042680B021A43426004E04268FF230133C0
:107630009A4342607047012904D142688B021A4381
:10764000426004E0426801239B029A434260704713
:10765000012904D14268CB021A43426004E0426827
:107660000123DB029A4342607047012904D142683A
:1076700002231A43426003E0426802239A434260B5
:107680007047012904D1426801231A43426003E094
:1076900042685208520042607047FF210131816008
:1076A0007047014688680122D2021040002801D0AC
:1076B000012070470020FCE70121C902816070476A
:1076C00001468868C007C00F002801D0012070471C
:1076D0000020FCE7F8B504460D46164600270DE0ED
:1076E000FBF76AFCE95D204600F048F800BF204641
:1076F000FFF7E6FF0028FAD0781C87B2B742EFDB2D
:107700000F48844201D10FA005E00F48844201D107
:107710000EA000E00DA001460EA000F087F80027A3
:1077200007E0FBF749FCE95D0DA000F07FF8781C4D
:1077300087B2B742F5DB0CA000F078F8F8BD000086
:107740000078014050430000006801405541525408
:10775000310000004D43552D3E25732000000000F0
:1077600030782530327820000D0A00000A46C168C2
:10777000090A0902D3B21943C1607047CA05D20D84
:1077800042617047012806D10649496A0122114326
:10779000044A516205E00349496A49084900014A1F
:1077A0005162704700F801400146064A506A0E23B4
:1077B00002469A4310460E220A401043014A506284
:1077C0007047000000F8014000B507484368180CF6
:1077D000D94389B2884203D1D8B200F019F802E047
:1077E0001F2000F015F800BD40FBFF1F012806D147
:1077F0000649496980221143044A516105E0034961
:10780000496980229143014A5161704700F8014063
:107810000146054A5069800980018A06920E10438C
:10782000014A50617047000000F801400FB410B5E4
:1078300003A9044B044A029800F00AF910BC08BCE2
:1078400004B018477D8A00003C0600200FB410B534
:1078500004A9074B02AA039800F0FAF8044602A90B
:10786000002000F091FC204610BC08BC04B0184772
:10787000898100002021020C01D010211046020A4B
:1078800001D010460839020901D01046091F8208AC
:1078900001D01046891E420801D0881E7047081A80
:1078A000704730B47446641E2578641CAB4204D320
:1078B000635D5B00E31830BC18471D46F8E702E043
:1078C00008C8121F08C1002AFAD17047704700206B
:1078D00001E001C1121F002AFBD17047F0B51FB4AF
:1078E00086B00998089A030D0021024314D051482C
:1078F000514A1818504305141198012810981AD0AD
:10790000281A401C00264D4F4D49009601910490C5
:10791000002812DA444211E01198012449A30128F9
:1079200001D11098C1430698119A84600360C26027
:1079300041600BB0F0BD4042E4E704462105002061
:107940003F4A001C51410391029012E0E00707D02A
:1079500032463B4601990098F8F702FE01910090EB
:1079600032463B4610461946F8F7FAFD06460F46E2
:107970006410002CEAD10498039B0028029A09990C
:10798000089806DAF8F7ECFD019B009AF8F7E8FD95
:1079900005E0F8F74DFE019B009AF8F749FE044612
:1079A0000E460022284BF8F75BFF03D80020C043A7
:1079B000014607E00022254B20463146F8F71EFD20
:1079C000F8F71AFF102409E0002C0ADB0A22002332
:1079D000F8F7BEFB079B30321A55641E02460A4375
:1079E000F2D11122641C079B121B1C19119B012B45
:1079F00003D0012308430ED10AE0084304D011202C
:107A000010900020119077E71098151A6D1E0BE06A
:107A10001098824202DD00236D1C03E0824201DAED
:107A200000236D1E002BEED0069811998260C16074
:107A300030C07EE701FCFFFF104D00000000144045
:107A40000000F03F300000000000F0430000E03F85
:107A5000FFB597B00646002518E2252877D1002407
:107A60002746FD49049400E00443761C3278012047
:107A7000203A90400842F7D130782A280ED00222CE
:107A8000307801463039092916D804990A23594318
:107A9000303940181443761C0490F1E7189802C856
:107AA00004911890002904DA01204003044348425D
:107AB000049002200443761C30782E2814D1042030
:107AC00004437078761C2A2809D11898761C80C83F
:107AD000189009E00A214F43303FC719761C3078CF
:107AE000014630390929F5D930786C2810D006DCE8
:107AF0004C281AD068280ED06A2817D104E07428C0
:107B000013D07A2812D110E00120400504430CE084
:107B10000121090501E0032109050C437178814227
:107B200003D1012000052418761C761C30781190B2
:107B300066280BD013DC58287DD009DC00287BD0C8
:107B40004528F6D04628F4D047281AD1A5E118E0F8
:107B5000632835D0642870D0652812D19DE1702843
:107B60006CD008DC6728F1D069287BD06E280DD056
:107B70006F2806D1BAE073282ED0752871D07828E6
:107B800059D01A9A199990476D1C7EE16002400FF6
:107B9000022809D003280DD00428189801680DD0B8
:107BA0000D60001D189070E11898EA1701680D60CB
:107BB0004A60F6E7189801680D80F2E70D70F0E76B
:107BC00018986A4601781172001D189000205072B2
:107BD00002A80090012005E0189802C81890002023
:107BE0000091C04361070DD5002101E00199491CB6
:107BF0000191B94212DA8142F8DB009A515C002906
:107C0000F4D10BE0002101E00199491C019181426E
:107C1000FADB019A0099895C0029F5D10199049851
:107C20001A9B471A21463846199A00F097FA01998B
:107C3000401945180BE04FE02CE113E04EE00098AE
:107C400000990078491C00911A9A19999047019857
:107C5000401E0190401CF2D1214638461A9B199AC9
:107C600010E137E00A200021009001916002410FED
:107C7000022907D0189A01CA1892C21794460329FC
:107C800008D00AE01898C01DC108C90005C918919C
:107C9000944607E000B2C2179446042902D140B2CC
:107CA000C1178C4600226146944506DA0A46002137
:107CB000404291418C462D2102E0210504D52B2123
:107CC0006A461173012103E0E10701D02021F7E7A3
:107CD000029155E00A200AE0102008E010200090F0
:107CE0000021042004430191082703E0082000211B
:107CF000019100906002410F022907D0189A01CA31
:107D0000189200229446032908D008E01898C01D54
:107D1000C108C90005C91891944603E080B204293E
:107D200000D1C0B200210291210729D511997029F3
:107D300006D0009A1021019B4A401A4305D00EE05C
:107D400040216A461173012108E06146014306D0D3
:107D500030216A4611731199517302210291009AE0
:107D60000821019B4A401A430AD16146014301D1CF
:107D7000610705D530216A46117301217F1E0291EA
:107D80001199582904D035A10E910DA90D910DE03E
:107D900037A1F9E76146019B009AF8F7D9F90E9BE4
:107DA0008C469B5C0D9A521E0D92137061460143E6
:107DB000F0D10D9805A9081A20300190600703D56D
:107DC00001200004844300E001270198874201DD7F
:107DD000381A00E000200199009041180298091813
:107DE0000498401A0490E00306D421461A9B199A7D
:107DF000049800F0B3F94519002706E003A81A9A81
:107E0000C05D199990476D1C7F1C02988742F5DB75
:107E1000E0030CD521461A9B199A049800F09EF9AC
:107E2000451904E01A9A3020199990476D1C009961
:107E3000481E00900029F5DC08E00D980D990078A7
:107E4000491C0D911A9A199990476D1C0199481E69
:107E500001900029F1DC63E109280100303132335F
:107E60003435363738396162636465660000000076
:107E70003031323334353637383941424344454660
:107E80000000000000F05AF94519761C30780028EF
:107E900000D0E2E528461BB0F0BD600700D40627FD
:107EA0001898C01DC108C90048680A680831C30F86
:107EB000DB071891190001D09CA108E0210501D52C
:107EC0009BA104E0E10701D09AA100E09AA1430040
:107ED00011985B08109165280CD006DC452809D064
:107EE00046281DD0472841D141E0662818D0672890
:107EF0003CD13CE00021112F01DB112000E0781C77
:107F00000191009008A911A8FFF7E8FC13990591C9
:107F10000021119A15927F1C12980197009150E050
:107F20000120C00703900120019008A9009711A823
:107F3000FFF7D4FC139A149905920022119B00922A
:107F400012981593059A0192002901D0104602E07B
:107F5000791C40180190381A01D5019804E040427C
:107F6000401E0090781C0190C01B029043E0012F3E
:107F700000DA01270021112F01DD112000E0384631
:107F80000191009008A911A8FFF7A8FC1399059189
:107F9000119A0021129815920091019721070CD493
:107FA0000599B94201DB019900E00191012904DD45
:107FB000159A491E515C302906D0B84201DA011DDC
:107FC00005DA0121029115E00199491EEDE700282B
:107FD00005DC0099411800910199091A03E0019A02
:107FE000411C914200DD01910099401A401C029011
:107FF0000120C0070390200706D40299019881420E
:1080000002DB0020C043029000206946C87707AF1A
:10801000012103980337C907884224D00220119018
:108020002B201290039800280CDA404203902D2058
:10803000129007E00A210398F8F760F830317F1EAC
:10804000039039701199481E11900029F2DC0398B1
:108050000028EFD1791E129808703078202108404E
:108060004530BF1E387006A8C01BC01D0390109875
:108070000078002800D00120019941180298C0170B
:108080000918039809180498401A401E0490E00348
:1080900006D421461A9B199A049800F05FF84519F6
:1080A00010980078002803D01A9A199990476D1CEF
:1080B000E00324D521461A9B199A049800F04EF843
:1080C00045191CE00098002807DB009905988842B4
:1080D00003DD1598405C199901E0199930201A9A2E
:1080E000904700986D1C401C00900298401E029022
:1080F000002804D11A9A2E20199990476D1C0199D5
:10810000481E01900029DDDC05E038781A9A7F1CB2
:10811000199990476D1C0399481E03900029F4DCBF
:1081200021461A9B199A0498ACE600002D00000025
:108130002B0000002000000000000000F8B50446FD
:1081400000251E461746880404D405E03946202041
:10815000B0476D1C641EF9D52846F8BDFFB504462E
:10816000002581B01E46C80301D5302700E0202736
:10817000880404D505E038460399B0476D1C641E99
:10818000F9D5284605B0F0BD0A68531C0B60107085
:1081900070470000F0B585B00446002004902248E6
:1081A000808AA0421ED22049898A601AF8F7B8FA5C
:1081B00000901E4801680098F8F7E2F801901C480A
:1081C00001680198F8F746F80746F8F735FB0546C9
:1081D0000022184BF8F7B6F903910290F8F754FB18
:1081E00004901DE01049898A081BF8F799FA00905D
:1081F0000E4801680098F8F7C3F801900C48016830
:108200000198F8F77CF80746F8F716FB05460022B8
:10821000084BF8F797F903910290F8F735FB0490B3
:10822000049805B0F0BD000040FBFF1F0C000020CB
:10823000100000200000E03FF0B587B004460027A2
:1082400013490A20085EF8F773FA05460022114B1D
:10825000F8F7EEF9039102900D4909896143084648
:10826000F8F77AFA054600220B4BF8F7E1F901918D
:108270000090039B029AF8F7C1F805910490F8F773
:1082800079FA0746002F00DA0027384607B0F0BD1C
:1082900080FAFF1F0000594000408F4010B50024B5
:1082A00000BFF8F711FD012801D1002010BD2046C4
:1082B000641C401C0028F4D10120F7E770B5044687
:1082C000606880470546E0784007400F002802DDDF
:1082D0002088401C2080E078C009A8421CD0E078AB
:1082E00038218843E1788906490F491CC9003822A2
:1082F00011400843E0708006400F032810DBE0784F
:1083000080218843E901802211400843E070E07831
:1083100038218843E07003E0E07838218843E0703A
:10832000E0784007400F0300FFF7BBFA0604285629
:10833000A7F4D1F4E078C009E1784906C90F884272
:1083400016D1A078F0218843A070A068002802D040
:108350002046A168884700202080A07800090001FD
:10836000401CA070E078C008C000401CE07004E031
:10837000A078F02188438030A070CBE0E078C0097D
:10838000E1784906C90F884212D0A078F0218843CD
:108390001030A070E068002802D02046E1688847CD
:1083A00000202080E078C008C000801CE07012E04F
:1083B000208864280FDDA078F02188435030A07019
:1083C000E069002802D02046E1698847E078C008CB
:1083D000C000401DE0709DE0E078C009E1784906EA
:1083E000C90F884220D1A078F0218843A070A068EE
:1083F000002802D02046A1688847A0780009000123
:10840000A178491C0907090F0843A07020690028BA
:1084100002D020462169884700202080E078C008EB
:10842000C000C01CE07027E020880F2824DDA07861
:108430000007000F01280BD1A078F02188433030CD
:10844000A0706069002813D02046616988470FE05A
:10845000A0780007000F02280AD1A078F0218843F5
:108460004030A070A069002802D02046A16988474A
:10847000E078C008C000E0704CE0E078C009E17826
:108480004906C90F88421AD0A078F02188431030DD
:10849000A070E068002802D02046E1688847208864
:1084A0000F2807DA00202080E078C008C000801C78
:1084B000E0700BE0E078C008C000E07006E02088C3
:1084C0000F2803DDE078C008C000E07022E0E0780B
:1084D000C009E1784906C90F88420BD1A078F02184
:1084E00088436030A070206A002812D02046216A9C
:1084F00088470EE0A078F02188431030A070E06833
:10850000002802D02046E1688847E078C008C00013
:10851000E07000BF00BF70BD10B50548046803E0FF
:108520002046FFF7CBFE646A002CF9D110BD000095
:10853000AC050020F7B584B0074616463B480068F6
:10854000039000253A4800680290002001903948C5
:108550000078002822D03848007800281ED13748FB
:10856000826928466D1C80003A5034484069441E98
:1085700033480068844211D33148006831490968A2
:108580004018A0420AD3102D08D20598854205D282
:1085900028466D1C80003C50012001902648007840
:1085A00000280CD00398864201D2039E07E002996E
:1085B00003984018B04202D20299039846182DE061
:1085C0003068041FE007C00F002800D125E03068A4
:1085D000441E1B480068001D84421DD318480068D3
:1085E000184909684018A04216D3102D14D2201F34
:1085F00000F0BCF900280FD0059885420CD2022D5E
:1086000006D10198002803D07868A04200D104E088
:1086100028466D1C80003C5000BF361D029903980F
:108620004018B042CCD8284607B0F0BDB0050020B5
:10863000B4050020C1050020C205002088190020D3
:10864000B8050020BC050020F0B58FB00E463546B9
:108650002C4620224D4907A8F7F7AAFD4C48076889
:108660004C48006806904C480078002809D14B4AD5
:108670004BA14DA0FFF7DAF853A0FFF7D7F800BFE2
:10868000FEE752480078002809D0444A50A146A08D
:10869000FFF7CCF84CA0FFF7C9F800BFFEE70120B8
:1086A0004A4908704DA0FFF7C1F847A0FFF7BEF890
:1086B00000F0D2F84A49C86AFFF7B8F842A0FFF7BD
:1086C000B5F82035BD4203D306983818A84202D227
:1086D0000120444908702A463846069900F064F99A
:1086E0004048007800284BD13D49086BFFF79EF8C1
:1086F00035A0FFF79BF83C49206808606068486037
:10870000A0688860E068C8602069086160694861A5
:10871000A0698861E069C8610846C068324A0A9960
:108720009268099B01930292039104902E4840683D
:1087300000902D48089B02682CA00799FFF776F857
:1087400021A0FFF773F82848C069274A0E9992695B
:108750000D9B01930292039104902348406900907D
:1087600021480C9B026921A00B99FFF75FF816A026
:10877000FFF75CF828A0FFF759F813A0FFF756F8A9
:10878000284600F01FFA0FB0F0BD000084950000ED
:10879000B0050020B4050020C00500207095000041
:1087A000696E69745F6F6B00282573292068617397
:1087B00020617373657274206661696C6564206101
:1087C000742025732E0000000D0A0000C105002052
:1087D000216F6E5F6661756C740000000000000020
:1087E000C4940000C20500208819002020202573B1
:1087F0003A2025303878202025733A2025303878E3
:10880000202025733A2025303878202025733A20FF
:1088100025303878000000003D3D3D3D3D3D3D3D6B
:108820003D3D3D3D3D3D3D3D3D3D3D3D3D3D3D3D78
:108830003D3D3D3D3D3D3D3D3D3D3D3D3D3D3D3D68
:108840003D3D3D3D3D3D3D3D3D3D3D3D3D3D3D3D58
:108850003D3D3D3D3D3D000010B50549054B064AF7
:1088600048680649FEF7E2FF05A0FEF7DFFF10BDEE
:10887000C4940000D8180020B818002098180020D0
:108880000D0A000010B504460C480068C02188435A
:108890000A49086008460068C02108430749086083
:1088A00007492046F7F72AFC064908700846007871
:1088B0007D21C90048430449088010BD00240040C0
:1088C00040420F0000000020020000200146114A33
:1088D00012884A43104B5A6100229A611A46126963
:1088E00001231A430C4B1A6100BF0B4A1069C207DF
:1088F000D20F002A04D0012212040240002AF4D030
:10890000054A126952085200034B1A6100229A610B
:10891000704700000200002000E000E00146114A1C
:1089200012784A43104B5A6100229A611A46126922
:1089300001231A430C4B1A6100BF0B4A1069C2078E
:10894000D20F002A04D0012212040240002AF4D0DF
:10895000054A126952085200034B1A6100229A61BB
:10896000704700000000002000E000E010B5014664
:108970000B884A881F20C00210401F24E402A04236
:1089800006D118400F242403A04201D1012010BDBC
:10899000FF200002104047242402A04201D1012000
:1089A000F5E70020F3E7000070B505460E461446D3
:1089B0001D48007800281CD01C480078002808D0EA
:1089C0001B4988692146FEF731FF1AA0FEF72EFFEA
:1089D00007E01749C8692146FEF728FF15A0FEF7F2
:1089E00025FFAC4201D22C4603E0A819A04200D2D8
:1089F000AC190F490869FEF719FF0EA0FEF716FF24
:108A000008E021460CA02268FEF710FF09A0FEF73F
:108A10000DFF241DA819A042F3D80EA0FEF706FFF3
:108A200004A0FEF703FF70BDC2050020C3050020AF
:108A3000C49400000D0A00002020616464723A2092
:108A40002530387820202020646174613A20253058
:108A5000387800003D3D3D3D3D3D3D3D3D3D3D3D8A
:108A60003D3D3D3D3D3D3D3D3D3D3D3D3D3D3D3D36
:108A70003D3D3D3D3D3D3D3D0000000070B504469F
:108A80000D46E1B20548FEF779FE00BF0348FEF748
:108A900017FE0028FAD0204670BD00000078014083
:108AA00010B5002823D0124B0022001F196803E0E4
:108AB000814203D80A4649680029F9D1002A0AD020
:108AC0001368841A9C4204D100681818106010467C
:108AD00002E0506000E01860002907D002680B1A1D
:108AE000934203D10B68D21802604968416010BDFF
:108AF0004006002001460148405C7047C2920000D9
:108B000001460148405C7047C291000010B5044620
:108B100021460548FEF732FE00BF0348FEF7D0FDB0
:108B20000028FAD010BD000000680140FEF7A6F949
:108B3000F8F7B2F9FEF716FBF8F726F9FAF754FA48
:108B400000F0E0FA00F0D6FAF8F734F9F8F74AFB4B
:108B500001E0FDF719FFFCE7F0B50B30C108C900D3
:108B6000144F0026144A0FE003688B420BD38B424C
:108B700005D95C1A4318456830C3083B00E04368D8
:108B8000136002C004E0021D10680028ECD13046DA
:108B9000002803D13868002801D00020F0BD064A23
:108BA00006481060064A121AD208D20044C00120BA
:108BB0003860D7E74406002040060020E42000206B
:108BC000E030002070B592B006460025402102A892
:108BD000F7F707FB3246102102A8FFF7ABFC05466A
:108BE000002410E0A10002AB5A58E1006118134BB9
:108BF000C81813A1FEF72AFE2021E0002018083033
:108C00000E4A1154641CAC42ECD3002D0DD00B481D
:108C1000E9006B180C4900900CA2086A0D49FEF798
:108C200005FE0DA0FEF702FE06E00749486AFEF7C2
:108C3000FDFD09A0FEF7FAFD12B070BDF818002086
:108C40002530386C78000000C49400002E617866EE
:108C500000000000981800200D0A000010B5FEF773
:108C6000FFF80A490968401A094988420BD9FEF7FA
:108C7000F7F806490860FF2101310648F9F7B1FC11
:108C800005A0FEF7D3FDFAF797F910BDB403002055
:108C9000581B0000C00C004063697263756C6174FE
:108CA000652074756E206F6E206C65640D0A00007F
:108CB00010B5FEF7D5F807490968401A06498842F9
:108CC00007D9FEF7CDF803490860F9F7BDFEFAF7BA
:108CD00073F910BDBC0300201027000010B5FAF78F
:108CE0006BF920212B48F9F76EFC002805D10821EB
:108CF00028484030F9F773FC04E00821254840304B
:108D0000F9F76BFCFAF714F9FAF7E2F80121890395
:108D10002048F9F758FC002806D00121C9031D4856
:108D2000F9F751FC002834D13220FFF7CFFD0121A3
:108D300089031848F9F747FC002816D116A0FEF75A
:108D400075FD802113484038F9F749FC402111484E
:108D50004038F9F744FCFF20F530FFF7B7FDFAF78C
:108D60002BF9FAF759F8F9F753FC0121C90309481F
:108D7000F9F729FC00280CD1F8F7C2FA3220FFF7E6
:108D8000A5FD01210348F9F728FCF9F769FBF9F77C
:108D90008DF810BD400D00405475726E5F4F6E200F
:108DA000706F77657220332E337620616E64207386
:108DB000656E6420677072730D0A000010B500F0D4
:108DC000E9F93A4908600846006839490968884263
:108DD00006D00520FFF77AFD00F0DCF93349086082
:108DE00032480068002808D031480068002804D1C3
:108DF000FEF736F82F49086051E02C48006800283B
:108E00004DD12B480068002849D0FEF729F82949A0
:108E10000968401A284908600846006827498842BE
:108E200016D20120F9F784F801280DD1C102244897
:108E3000F9F7D5FB0121C9032148F9F7D0FB01213E
:108E400049031F48F9F7CBFB1EA0FEF7EFFC26E015
:108E5000194800687D218901884208D216480068B7
:108E60004910884203D91DA0FEF7E0FC17E0124824
:108E700000687D218901884211D31EA0FEF7D6FC2F
:108E80000121C9020E48F9F7AAFB012189030C4808
:108E9000F9F7A5FB012149030948F9F7A0FBFAF707
:108EA0008BF8024800680249086010BDCC0300201E
:108EB000D0030020C4030020C8030020C409000020
:108EC000400C004053686F72742070726573732099
:108ED00064657465637465642E0A00006C6F6E6768
:108EE0002070726573732064657465637465642EA5
:108EF0000A0000004C6F6E67206C6F6E6720707206
:108F00006573732064657465637465642E0A00007C
:108F100010B50820F9F70CF8002818D1002414E047
:108F2000FF2101312E48F9F758FBFF20F530FFF7FC
:108F3000CDFCFF2101312A48F9F751FBFF20F53024
:108F4000FFF7C4FCFAF738F8641C032CE8DB0821AF
:108F500023488038F9F737FB002805D10421204841
:108F6000C038F9F73CFB04E004211D48C038F9F78C
:108F700034FB04211A488038F9F725FB002805D175
:108F800002211748C038F9F72AFB04E002211448EF
:108F9000C038F9F722FB0820F8F7CAFF002805D1EE
:108FA00001210F48C038F9F71AFB04E001210C48F1
:108FB000C038F9F712FB012149030948C038F9F715
:108FC00002FB002805D108210548C038F9F707FB46
:108FD00004E008210248C038F9F7FFFA10BD00008C
:108FE000C00C004070B5F9F7E7FFFDF739FF2749DE
:108FF0000968401A2649884247D9FDF731FF2349BD
:109000000860F9F737FC04462249F7F71AF9F9F72F
:1090100081FC04461F49091FF7F713F9F9F7CAFC49
:109020001D4908601B48F7F702F90646F7F704FCEC
:10903000044622460B4619A0FEF7F8FB1548001F10
:10904000F7F7F5F80646F7F7F7FB044622460B4616
:1090500017A0FEF7EBFB10480068F7F7EDFB04469E
:1090600022460B4617A0FEF7E1FB0120F8F760FF50
:10907000002802D119A0FEF7D9FB0120F8F758FF0C
:10908000002802D118A0FEF7D1FB70BDB803002064
:109090001027000001010020D4030020616C6B61E7
:1090A00020766363203D252E32660D0A0000000005
:1090B0006C69746820766363203D20252E3266201B
:1090C0000D0A00006D63755F74656D706572617483
:1090D00075726520252E31660D0A0000616C6B618A
:1090E000206C6F73650D0A006C697468206C6F7377
:1090F000650D0A0010B5FDF71AF9FAF763FDFAF7E6
:10910000DFFB10BDFEB500201E4908607D24E40091
:109110002046604301461C48F6F7F0FF0546294605
:109120002046FDF76DFF002705E00120FFF7CEFB8D
:10913000F9F742FF7F1C7D20C0008742F5D3002055
:10914000F8F7DEF80F4806686E432046F7F7E8FAAE
:1091500007463046F7F7E4FA39460090F7F7D3F8B8
:1091600002900A490298F7F7C6F808490090F7F705
:1091700007F907460649F7F7C6F801900120F8F706
:10918000BFF8FEBDB0030020001BB700001B374B2B
:109190000000C84210B5012149020448F9F713FA4A
:1091A000002801D1012010BD0020FCE7000D004087
:1091B000014648000A06D20F1B235A435040C0B252
:1091C0007047637C777BF26B6FC53001672BFED7EE
:1091D000AB76CA82C97DFA5947F0ADD4A2AF9CA440
:1091E00072C0B7FD9326363FF7CC34A5E5F171D8B0
:1091F000311504C723C31896059A071280E2EB279E
:10920000B27509832C1A1B6E5AA0523BD6B329E3C0
:109210002F8453D100ED20FCB15B6ACBBE394A4CA0
:1092200058CFD0EFAAFB434D338545F9027F503C20
:109230009FA851A3408F929D38F5BCB6DA2110FF4C
:10924000F3D2CD0C13EC5F974417C4A77E3D645D49
:10925000197360814FDC222A908846EEB814DE5ED6
:109260000BDBE0323A0A4906245CC2D3AC6291952A
:10927000E479E7C8376D8DD54EA96C56F4EA657A66
:10928000AE08BA78252E1CA6B4C6E8DD741F4BBD07
:109290008B8A703EB5664803F60E613557B986C1B4
:1092A0001D9EE1F8981169D98E949B1E87E9CE55D1
:1092B00028DF8CA1890DBFE6426841992D0FB0547B
:1092C000BB1652096AD53036A538BF40A39E81F33C
:1092D000D7FB7CE339829B2FFF87348E4344C4DE67
:1092E000E9CB547B9432A6C2233DEE4C950B42FA57
:1092F000C34E082EA16628D924B2765BA2496D8B95
:10930000D12572F8F66486689816D4A45CCC5D65A5
:10931000B6926C704850FDEDB9DA5E154657A78DD0
:109320009D8490D8AB008CBCD30AF7E45805B8B341
:109330004506D02C1E8FCA3F0F02C1AFBD030113DB
:109340008A6B3A9111414F67DCEA97F2CFCEF0B4C5
:10935000E67396AC7422E7AD3585E2F937E81C7503
:10936000DF6E47F11A711D29C5896FB7620EAA1801
:10937000BE1BFC563E4BC6D279209ADBC0FE78CD90
:109380005AF41FDDA8338807C731B112105927805E
:10939000EC5F60517FA919B54A0D2DE57A9F93C9FD
:1093A0009CEFA0E03B4DAE2AF5B0C8EBBB3C83532D
:1093B0009961172B047EBA77D626E169146355218B
:1093C0000C7D8D01020408102040801B366CD8AB48
:1093D0004D9A2F5EBC63C697356AD4B37DFAEFC54C
:1093E000913972E4D3BD61C29F254A943366CC8320
:1093F0001D3A74E8CB8D01020408102040801B3612
:109400006CD8AB4D9A2F5EBC63C697356AD4B37DDA
:10941000FAEFC5913972E4D3BD61C29F254A9433F6
:1094200066CC831D3A74E8CB8D01020408102040FD
:10943000801B366CD8AB4D9A2F5EBC63C697356ADD
:10944000D4B37DFAEFC5913972E4D3BD61C29F25D3
:109450004A943366CC831D3A74E8CB8D010204082C
:10946000102040801B366CD8AB4D9A2F5EBC63C673
:1094700097356AD4B37DFAEFC5913972E4D3BD61F3
:10948000C29F254A943366CC831D3A74E8CB8D0184
:10949000020408102040801B366CD8AB4D9A2F5E1A
:1094A000BC63C697356AD4B37DFAEFC5913972E4CF
:1094B000D3BD61C29F254A943366CC831D3A74E8BC
:1094C000CB0000006497000054960000D89700007D
:1094D000BC970000C0950000E8950000649B000068
:1094E000809B000084960000F09700002097000009
:1094F00000970000109600008C980000D49800009F
:1095000004980000BC99000084990000E49A0000CF
:10951000909A00003C9A0000649A0000409B000072
:109520001C9B0000B49A00000C9900003C970000BE
:109530006498000034990000949700009C9B000000
:10954000189A0000B0980000409800006099000050
:10955000F4990000E0960000C4960000636D5F621D
:1095600061636B74726163655F61737365727400CC
:10957000636D5F6261636B74726163655F66617581
:109580006C740000A4950000A8950000AC95000044
:10959000B0950000BC950000B8950000B49500009F
:1095A00050960000523020005231200052322000EC
:1095B00052332000504320004C52200052313200E0
:1095C0003D3D3D3D3D3D3D3D3D3D3D20CFDFB3CCAF
:1095D000B6D1D5BBD0C5CFA2203D3D3D3D3D3D3DA3
:1095E0003D3D3D3D000000003D3D3D3D3D3D3D3D9F
:1095F0003D3D3D3D20D6F7B6D1D5BBD0C5CFA2204D
:109600003D3D3D3D3D3D3D3D3D3D3D3D000000007E
:109610003D3D3D3D3D3D3D3D3D3D3D3D3D3D3D3D7A
:109620003D3D3D3D3D3D3D3D3D20BCC4B4E6C6F71E
:10963000D0C5CFA2203D3D3D3D3D3D3D3D3D3D3D65
:109640003D3D3D3D3D3D3D3D3D3D3D3D3D3D0000C4
:1096500050535200B9CCBCFEC3FBB3C6A3BA2573AA
:10966000A3ACD3B2BCFEB0E6B1BEBAC5A3BA2573F3
:10967000A3ACC8EDBCFEB0E6B1BEBAC5A3BA2573B3
:1096800000000000B2E9BFB4B8FCB6E0BAAFCAFD52
:10969000B5F7D3C3D5BBD0C5CFA2A3ACC7EBD4CB52
:1096A000D0D0A3BA61646472326C696E65202D6596
:1096B0002025732573202D61202D6620252E2A73E9
:1096C00000000000B7A2C9FAD7DCCFDFB4EDCEF3BB
:1096D000B5C4B5D8D6B7A3BA253038780000000095
:1096E000B7A2C9FAB4E6B4A2C6F7B9DCC0EDB4EDCE
:1096F000CEF3B5C4B5D8D6B7A3BA253038780000B4
:10970000D4DAD6D0B6CFBBF2C2E3BBFABBB7BEB396
:10971000CFC2B7A2C9FAB4EDCEF3D2ECB3A3000026
:10972000D4DACFDFB3CC28257329D6D0B7A2C9FAB3
:10973000B4EDCEF3D2ECB3A300000000B7A2C9FA97
:10974000D3C3B7A8B4EDCEF3A3ACD4ADD2F2A3BAD1
:10975000CAD4CDBCC7D0BBBBB5BD2041524D20D76C
:10976000B4CCAC00B4EDCEF3A3BACEDEB7A8BBF157
:10977000C8A1D6F7D5BBD0C5CFA2A3ACC7EBBCEC74
:10978000B2E9D6F7D5BBB5C4CFE0B9D8C5E4D6C3E6
:1097900000000000B7A2C9FAD3C3B7A8B4EDCEF356
:1097A000A3ACD4ADD2F2A3BAC6F3CDBCD6B4D0D05C
:1097B000B7C7B6D4C6EBB7C3CECA0000D4DAD6D08A
:1097C000B6CFBBF2C2E3BBFABBB7BEB3CFC2B7A240
:1097D000C9FAB6CFD1D40000D4DACFDFB3CC282574
:1097E0007329D6D0B7A2C9FAB6CFD1D400000000F1
:1097F000BBF1C8A1BAAFCAFDB5F7D3C3D5BBCAA7E1
:10980000B0DC0000B7A2C9FAB4E6B4A2C6F7B9DC6E
:10981000C0EDB4EDCEF3A3ACD4ADD2F2A3BAC6F38F
:10982000CDBCB4D3B2BBD4CAD0EDB7C3CECAB5C4D5
:10983000C7F8D3F2B6C1A1A2D0B4CAFDBEDD000004
:10984000B7A2C9FAB5F7CAD4B4EDCEF3A3ACD4AD80
:10985000D2F2A3BACAFDBEDDBCE0B2E2B5E3C6A552
:10986000C5E40000B7A2C9FAD3C3B7A8B4EDCEF3DC
:10987000A3ACD4ADD2F2A3BACEDED0A7B5C4D2EC9D
:10988000B3A3B7B5BBD8C2EB00000000B7A2C9FABA
:10989000D3B2B4EDCEF3A3ACD4ADD2F2A3BAC8A187
:1098A000D6D0B6CFCFF2C1BFCAB1B3F6B4ED000087
:1098B000B7A2C9FAB5F7CAD4B4EDCEF3A3ACD4AD10
:1098C000D2F2A3BAD6B4D0D020424B505420D6B84E
:1098D000C1EE0000B7A2C9FAB4E6B4A2C6F7B9DC7B
:1098E000C0EDB4EDCEF3A3ACD4ADD2F2A3BAC6F3BF
:1098F000CDBCB4D3B2BBD4CAD0EDB7C3CECAB5C405
:10990000C7F8D3F2C8A1D6B8C1EE0000B7A2C9FA11
:10991000D3C3B7A8B4EDCEF3A3ACD4ADD2F2A3BAFF
:10992000C6F3CDBCD6B4D0D0CEB4B6A8D2E5D6B8A6
:10993000C1EE0000B7A2C9FAD3C3B7A8B4EDCEF305
:10994000A3ACD4ADD2F2A3BAC6F3CDBCD6B4D0D0BA
:10995000D0ADB4A6C0EDC6F7D6B8C1EE0000000089
:10996000B7A2C9FAB5F7CAD4B4EDCEF3A3ACD4AD5F
:10997000D2F2A3BAB7A2C9FACFF2C1BFB2B6BBF155
:1099800000000000B7A2C9FAB4E6B4A2C6F7B9DC79
:10999000C0EDB4EDCEF3A3ACD4ADD2F2A3BAC8EB14
:1099A000D5BBCAB1C6F3CDBCB7C3CECAB2BBB1BB7F
:1099B000D4CAD0EDB5C4C7F8D3F20000B7A2C9FA33
:1099C000B4E6B4A2C6F7B9DCC0EDB4EDCEF3A3ACF7
:1099D000D4ADD2F2A3BAB3F6D5BBCAB1C6F3CDBCEF
:1099E000B7C3CECAB2BBB1BBD4CAD0EDB5C4C7F8F9
:1099F000D3F20000B7A2C9FAB5F7CAD4B4EDCEF3DA
:109A0000A3ACD4ADD2F2A3BACDE2B2BFB5F7CAD4FB
:109A1000C7EBC7F300000000B7A2C9FAB5F7CAD474
:109A2000B4EDCEF3A3ACD4ADD2F2A3BA4E564943B3
:109A300020CDA3BBFAC7EBC7F3000000B7A2C9FA59
:109A4000D7DCCFDFB4EDCEF3A3ACD4ADD2F2A3BA62
:109A5000BEABC8B7B5C4CAFDBEDDD7DCCFDFB4ED41
:109A6000CEF30000B7A2C9FAD7DCCFDFB4EDCEF356
:109A7000A3ACD4ADD2F2A3BAB2BBBEABC8B7B5C427
:109A8000CAFDBEDDD7DCCFDFB4EDCEF300000000B1
:109A9000B7A2C9FAD7DCCFDFB4EDCEF3A3ACD4AD17
:109AA000D2F2A3BAD6B8C1EED7DCCFDFB4EDCEF395
:109AB00000000000B7A2C9FAD7DCCFDFB4EDCEF3C7
:109AC000A3ACD4ADD2F2A3BAB6E8D0D4B1A3B4E675
:109AD000B8A1B5E3D7B4CCACCAB1B7A2C9FAB4ED5A
:109AE000CEF30000B7A2C9FAB4E6B4A2C6F7B9DC57
:109AF000C0EDB4EDCEF3A3ACD4ADD2F2A3BAB6E8C8
:109B0000D0D4B1A3B4E6B8A1B5E3D7B4CCACCAB154
:109B1000B7A2C9FAB4EDCEF300000000B7A2C9FAAB
:109B2000D7DCCFDFB4EDCEF3A3ACD4ADD2F2A3BA81
:109B3000C8EBD5BBCAB1B7A2C9FAB4EDCEF30000E9
:109B4000B7A2C9FAD7DCCFDFB4EDCEF3A3ACD4AD66
:109B5000D2F2A3BAB3F6D5BBCAB1B7A2C9FAB4ED73
:109B6000CEF30000B4EDCEF3A3BACFDFB3CCD5BBB8
:109B7000282530387829B7A2C9FAD2E7B3F6000011
:109B8000B4EDCEF3A3BAD6F7D5BB28253038782963
:109B9000B7A2C9FAD2E7B3F600000000B7A2C9FA2B
:109BA000D3C3B7A8B4EDCEF3A3ACD4ADD2F2A3BA6D
:109BB000C6F3CDBCD6B4D0D0B3FD203020B2D9D7B7
:109BC000F7000000E49B00000000002048060000B1
:109BD000A00A0000249E000048060020986A0000A9
:109BE000CE780000417205259632B8411AF004176C
:109BF000784D55ECDC2517276C5169AA26123C14C8
:109C000001A0051310010216101A0A31110009A152
:109C100008070605040302017208BB0101AC826457
:109C200085D002D0020916CE16200102603F137FB4
:109C3000068E0832011F060E1A305452102344803B
:109C40001303021328011320634A050912014A086D
:109C500009214A090912034A0B09227012023A2A01
:109C60001B4A010912954A04092A963F29091297AD
:109C70004A06092A9036290912914A0C0912924A79
:109C80000D0912934A0E0912944A0F09198F1202F4
:109C90001A2C092A115A290912124A02092A13A256
:109CA00029092A146C29092A156C29092A05AB29C6
:109CB00009199112021A2E092A213F29092A223F45
:109CC00029092A233F29092A243F29092A303F2923
:109CD000092A31AB290912324A07092A25512909D3
:109CE0002A26FC290912274A0A092A28CF29092AE3
:109CF00029CF29092A41751A30092A427529092ACA
:109D0000437529092A447529092A457529092A46CE
:109D10007529092A477529092A407529092A48758C
:109D200029092A497529092A507529092A517529AD
:109D3000092A666C1A32092A066C29092A336C2909
:109D4000092A606C29092A616C29092A626C29098F
:109D50002A656C29092A646C29092A716C2909422F
:109D6000011A34091202190B29091A03623909125E
:109D7000044A030912054A040912064A080912078F
:109D80004A090912084A0A0912094A0B09120A4A21
:109D90000C09012C169901030DADA40E5743195857
:109DA000521E2AB499B904214B5816605AA8085A71
:109DB000D0085AF808016E0334803FA40A341248D0
:109DC0000F5546473232304731304C4E565A2001FB
:109DD000011414202301021D1040096666664166C5
:109DE0006686410809109A999941CDCCCC3DAB23A8
:109DF00002431A08044B8C42042910690CC92C1226
:109E000028123216F6FFF1FF2854F1FF321A320AF7
:109E1000811A640E41199449696961012603670139
:049E200001D3127ADE
:04000005000000C136
:00000001FF
